:1079F90053797374656D436C6F636B3A20384D48E6
:107A09007A000D0A425354415455533A25780D0AC8
:017A1900006C
:0E7CDF00C29CD2A08F993099FDC2A0C29922FA
:105D8800126EAC7BFF7A7979F9122C8E3070205321
:105D9800B1F8C270127BA0127D05127A3A127634DD
:105DA800126DC41270B912784512611D127B6030F1
:105DB8006F32B2A47BFF7A7A790B9002A5E0900249
:105DC800BDF0122C8EC26F122559126634127AEA6F
:105DD800127A77127A941265694003125976127B07
:105DE8008B124DEB127872127AB1126C391250453F
:105DF8001256D2900206E524F0A3E525F0A3E52289
:085E0800F0A3E523F0808522E0
:1073C4009005367401F07E027F3C7B40E4FD127828
:1073D400C97E027F0A7B14E41278C9900224740ADD
:1073E400F0A374ABF0A3740AF0A374ABF0C22CC284
:1073F4002D9003FF7402F0D22ED27E90027C745042
:02740400F02274
:105976007FFE7E011278F3501F7B007A02E4FDFC65
:10598600FFFE1267B47FFE7E031278F3402CE4FD1F
:10599600FF7E02125B4A80227FFE7E031278F3505E
:1059A600167B007A02E4FDFCFF7E021267B4E4FD7A
:1059B600FFFE125B4A8003D27122900000E0F520C0
:1059C600A3E0F521900238E520F0A3E521F0900050
:1059D6001A12241E90022C122484900022E0FFA3A7
:1059E600E0900236CFF0A3EFF0E52154072403F54B
:1059F6001364056005E513B40A04E4F51422E513FF
:105A060064046005E513B4090475140122751402D3
:015A1600226D
:107A5900C2AFD2ACC086758640C28FD086D2AD4344
:0E7A6900BA6043E840E4F5D843A908D2AF2242
:10789E007580F075E18F75E9C075908075E27F7522
:1078AE00EA8075A04675E3BB75EB4675B01875E4B6
:0B78BE00E675EC184380C043E980220F
:106EAC00E4FF1279D712789E1259761273C47D05BD
:106EBC007C007F44127815126695127B337D647FBB
:106ECC00A07E0F12601F125E97125E104002D25D00
:106EDC001275823007121260A04002D2397E047FF4
:0C6EEC0097125C6F4002D27B127A592290
:10102E00EFB4200E206603306919E4FF1279D7D28F
:10103E006822EFB4400D206603306907E4FF127991
:04104E00D7D268226B
:1079B300D26E90049FE004F0C3940A4004E4F0D232
:1079C3007090049EE004F0C394C84004E4F0D26FC6
:0479D3001258D42250
:1074C700D3EF9450EE940040037F0522D3EF943C12
:1074D700EE940040037F0422D3EF9428EE940040FB
:1074E700037F0322D3EF9414EE940040037F02221C
:0F74F700D3EF9400EE940040037F01227F002228
:107BB40030740F90053EE004F0C394644004E4F094
:037BC400C2742266
:10687000302A1490053CE004F0C3940A400BE4F085
:10688000A2B5B392B58002C2B530750D90053DE05A
:1068900004F0C394054002E4F030742C900234E01C
:1068A000FEA3E0FF1274C7EF6401601CEFB40204A2
:1068B000D2A18014EFB40306D2A1D2A2800AEFB411
:0B68C0000406D2A1D2A2D2A3127BB426
:0168CB0022AA
:10650300C22CC22DC22E302B569003FFE07018040C
:10651300F0D22D900089E0FEA3E0FF90008CE0FD17
:1065230012601F43B701229003FFE0B40116740207
:10653300F0D22E900089E0FEA3E0FF7D6412601F7D
:1065430043B70122E49003FFF0D22C900089E0FED0
:10655300A3E0FF90008BE0FD12601F43B70122C24E
:066563002CC22DC22E2205
:1077E500307D2CC27DE50824FE600F24F16016145F
:1077F50060102411701912650322D274E490053EBD
:10780500F022D26622B275307503C28322D283225A
:1074470030683CC268306924E4FF1279D7D2AFC2F2
:1074570069E49005E8F07F011271DAD2ACD2ADD2BF
:10746700CE7F70127B1C127C85127C13E49005E89A
:10747700F0A3F09003F7F09003F8F09003F9F022EF
:107CAB0053B1F8C2AFD283E4FF127B7612794180D5
:027CBB00EF22B6
:1076A900D283C275127C26127C987F70127CBDC26F
:1076B900CE53B77E302904D2A58002C2A57F01121C
:1076C90071DAC2AFC2ACC2ADE4F5D87F801279D706
:0676D900D2AF127CF92281
:105BE10030670E204306204403304505C267D26664
:105BF1002230161490002AE0FF9005E9E004F0C37A
:105C01009F406AEFF0D2662220745B202A50202B3D
:105C11004D30191490002AE0FF9005E9E004F0C32B
:105C21009F404AEFF0D26622E49005E9F0A2127299
:105C3100107218721A721172137219721B721C721D
:105C4100157275401390002AE0FF9005E8E004F01A
:105C51009F401AEFF0D26922E49005E8F022E49027
:0E5C610005E8F0A3F022E49005E8F0A3F0229D
:10748700206926206623C2AFA27C727D7272726861
:10749700724C7270726F400D9005EAE064126005DD
:1074A700D2AF127CEDD2AF801330660AD27212507F
:1074B70045127CAB80063069031276A91274472205
:10710200000000300062007400000089008E0099C7
:1071120000A200AA00BB00BF00FE000000000000A9
:10712200000000000020005000820094000000A92E
:1071320000AE00B900C200CA00DB00DF011E000081
:08714200000000000000000045
:107B4A00900402E07008C29C75995AD2A022C29C85
:067B5A007599FFD2A02284
:086193009002B8EEF0A3EFF05A
:10619B007B017A047900900402E02403FD127ACE8D
:1061AB00900402E02403F582E43404F583E06F707D
:1061BB0043FF900402E0FEEFC39E502953B1F874E5
:1061CB00032FF582E43404F583E0FE9002B8E0FC83
:1061DB00A3E0F5828C83EEF09002B8E475F0011227
:1061EB0022480F80CDD273E49005F5F0C29C7599CF
:0B61FB005AD2A022C29C7599FFD2A0CE
:016206002275
:1065CF00900402E0D3948C4002E4F0E4FD900402C6
:1065DF00E0FCEDC39C501D53B1F88F828E83E0FB1E
:1065EF0074032DF582E43404F583EBF00FBF000143
:1065FF000E0D80D97B017A047900EC2403FD127A09
:10660F00CE900402E02403F582E43404F583EFF026
:10661F00C29C9003FAE02400F582E43404F583E091
:04662F00F599D2A067
:016633002244
:107070007B017A047900900402E02403FD127ACEA9
:10708000900402E02403F582E43404F583E0B507BC
:1070900020900404E0FFB441089005EA7412F080E7
:1070A00006EFB40502D267C243C29C75995AD2A0BA
:0970B00022C29C7599FFD2A022B6
:1075BE007B017A047900900402E02403FD127ACE56
:1075CE00900402E02403F582E43404F583E0B50769
:1075DE0012900403E09003F2F0C243C29C75995AD4
:0B75EE00D2A022C29C7599FFD2A022FF
:1043C200900401E0FF122506441601441602441629
:1043D20003441604441605441606441607441608F8
:1043E20044160944160A44270B44370C443F0D4433
:1043F200470E444F0F442F10445711445F12446735
:1044020013446F14447715447F16448717448F185A
:1044120000004497EF25E02408F582E43402AF82DD
:10442200FE1265CF227E027F1E1265CF227E027FA0
:10443200201265CF227E027F241265CF227E027F68
:10444200261265CF227E027F281265CF227E027F4E
:104452002A1265CF227E027F2C1265CF227E027F36
:10446200301265CF227E027F341265CF227E027F18
:10447200361265CF227E027F061265CF227E027F30
:10448200081265CF227E027F381265CF227E027F1C
:104492003A1265CF22900402E0C394804009D23AD6
:1044A2009003E27401F022900401E0B478109003CA
:1044B200F2E0B40C09D23A9003EF7401F0229004B6
:1044C20001E0B478229003F2E025E02402F582E4D0
:1044D2003471F583E493FE740193FF9002B6EEF01B
:1044E200A3EFF01265CF22900401E0B4792190038A
:1044F200F2E025E02426F582E43471F583E493FEAC
:0F450200740193FF9002B6EEF0A3EFF01265CFB5
:014511002287
:106AE7007B017A047900900402E02403FD127ACE38
:106AF700900402E02403F582E43404F583E06F7028
:106B07002F900403E0FEA3E0FDEEEDFF9005DFEE1E
:106B1700F0A3EFF04E7008C29C7599FFD2A022D265
:106B27007C9005DAE04401F0C29C75995AD2A02204
:086B3700C29C7599FFD2A02257
:104F82007B017A047900900402E02403FD127ACEB8
:104F9200900402E02403F582E43404F583E06F60B8
:104FA2000302503D900404E0FFE4FCFDFE78101281
:104FB20023FFC004C005C006C007900403E0FFE45D
:104FC200FCFDFE78181223FFD003D002D001D000DE
:104FD200122396C004C005C006C007900405E0FF76
:104FE200E4FCFDFE78081223FFD003D002D001D0EA
:104FF20000122396A804A905AA06AB07A3E0FFE4C2
:10500200FCFDFE1223969005D61224849002A1E0A4
:105012007002A3E0600C9005D612241EEC4D4E4F98
:105022007008C29C7599FFD2A022D27C9005DAE06A
:105032004410F0C29C75995AD2A022C29C7599FF65
:03504200D2A022D7
:10766F007B017A047900900402E02403FD127ACEA4
:10767F00900402E02403F582E43404F583E0B507B7
:10768F0011D27C9005DAE04420F0C29C75995AD251
:0A769F00A022C29C7599FFD2A02220
:106E12007B017A047900900402E02403FD127ACE09
:106E2200900402E02403F582E43404F583E06F70F9
:106E320024D27C900403E0FEA3E0FDEEEDFF90057A
:106E4200DBEEF0A3EFF09005DAE04404F0C29C75AB
:0D6E5200995AD2A022C29C7599FFD2A022AD
:106E5F007B017A047900900402E02403FD127ACEBC
:106E6F00900402E02403F582E43404F583E06F70AC
:106E7F0024D27C900403E0FEA3E0FDEEEDFF90052D
:106E8F00DDEEF0A3EFF09005DAE04408F0C29C7558
:0D6E9F00995AD2A022C29C7599FFD2A02260
:106B3F007B017A047900900402E02403FD127ACEDF
:106B4F00900402E02403F582E43404F583E06F70CF
:106B5F002FFF74032FF582E43404F583E0FE74E114
:106B6F002FF582E43405F583EEF00FEFB407E3D28F
:106B7F007C9005DAE04480F0C29C75995AD2A0222D
:076B8F00C29C7599FFD2A022
:016B960022DC
:10577E00900401E012250657AA1857AE7757CA783B
:10578E0057EC7957B6A057BEA157C2A257B2A3572E
:10579E00BAA457C6AF580EB0000058281270702227
:1057AE001275BE22124F8222126AE72212766F22E1
:1057BE00126E1222126E5F22126B3F229003F2E0E3
:1057CE0025E02402F582E43471F583E493FE74013E
:1057DE0093FF9002B6EEF0A3EFF0126193229003C6
:1057EE00F2E025E02426F582E43471F583E493FE9D
:1057FE00740193FF9002B6EEF0A3EFF012619322C4
:10580E00900403E0B4550CD23AD238C29C75995A22
:0A581E00D2A022C29C7599FFD2A00F
:01582800225D
:1040F100E49002B6F0A3F09003FAE0FFB4021A9044
:104101000401E064A56006E49003FAF022E4900360
:10411100FDF0A3F09003F3F022900402E0FD7C0097
:104121002409FBEC33FA7E00C3EF9BEA6480F87448
:104131008098505FED2407FDEC33FCD3EF9DEC64D8
:1041410080F874809850189003FAE024FFF582E417
:104151003403F583E0FF9003FDEE8FF012224890C7
:1041610003FAE0FFB40511900404E0640770030250
:104171004259E49003FAF022EF64066003024259C7
:10418100900405E0640670030242599003F3E04491
:1041910020F022E49003FAF0900402E0FD2408F5F7
:1041A10082E43404F583E0FE74072DF582E43404DF
:1041B100F583E07C002400FFEC3EFE9003FDE06E01
:1041C1007003A3E06F60079003F3E04480F0900375
:1041D100F3E0FF6006900406F08007D24CE49004FF
:1041E10006F0E4900402F0900405740BF0900403CF
:1041F100E0FFA3E0900403F0A3EFF07F029004023C
:10420100E0FE2407FDE433FCEFC39DEC6480F87409
:104211008098501874002FF582E43404F583E0FD92
:104221009002B6E48DF01222480F80D19002B6E0E0
:10423100FCA3E0FF74072EF582E43404F583EFF06C
:10424100ECFF900402E02408F582E43404F583EFE6
:08425100F0C29C75995AD2A03D
:014259002242
:105AB3009003FAE02400F582E43404F583EFF090D8
:105AC30003FAE004F0E0C3948C4002E4F09003FA9C
:105AD300E064017027900400E0FF54FEB59A10EFD4
:105AE30020E006D246C2498013D249C246800D90B7
:105AF3000400E0645A6005E49003FAF030460D9028
:105B030003FAE0640370301243C2802B30492590BE
:105B13000402E02403FFE433FE9003FAE0D39FEE94
:105B23006480F8748098400F12577EC249E4900352
:105B3300FAF080031240F1C243E49005E8F09005C7
:075B4300E9F09003F7F022E6
:10556C00900400E0B45A06A3E064A56003304C48F4
:10557C00900402E02408FFE433FE9003FAE0C39F9A
:10558C00EE6480F87480984016D29CC2A0E4F0C2FD
:10559C0046900400F0A3F0A3F0A3F0D243806690F1
:1055AC0003FAE004F0C29CE02400F582E43404F534
:1055BC0083E0F599D2A0804D9003FAE0FF6016903D
:1055CC000402E02403FDE433FCC3EF9DEC6480F89B
:1055DC007480984019D29CC2A0E49003FAF0C246A1
:1055EC00900400F0A3F0A3F0A3F0D2438017900333
:1055FC00FAE004F0C29CE02400F582E43404F58364
:10560C00E0F599D2A0E49005E8F09005E9F090035C
:03561C00F7F02282
:107B60009003F7E004F0C39404400AE4F09003FAB1
:067B7000F0D29CC2A0222D
:107AEA00305F119002B1E004F0C39405400BD25DFF
:0A7AFA007405F022E49002B1F022BE
:0E5829009002C1EFF0A3EDF0A3EAF0A3EBF0C4
:10583700C24EE4A3F0305D030258CCA3F09002C23D
:10584700E0FF9002C6E0C39F507B9002C5E0FF04D3
:10585700F0EFC39405503E9002C1E0FD7C0090023A
:10586700FA7401F0A3F09002C3E0FFA3E09002FCFA
:10587700CFF0A3EFF0E4FB7F36124512924E304E85
:1058870004801280C5E4F5C87F011271DA127B33F8
:105897001271DA80B59002C5E0C3940540048025F3
:1058A7008015E49002C5F09002C1E004F09002C3B5
:1058B700E475F0011222487F011271DA9002C6E006
:0C58C70004F0025844A24EB3925FA24EBF
:0158D30022B2
:0E642D009002C4EFF0A3EDF0A3EAF0A3EBF0B1
:10643B00C24EE4A3F0205D4D9002C8E0FF04F0EFE4
:10644B00C3940550409002C4E0FD7C00A3E0900291
:10645B00F0F0A37401F09002C6E0FFA3E09002F20B
:10646B00CFF0A3EFF0E4FB7F36123A95924E304E0D
:10647B0004801280C3E4F5C87F011271DA127B33FA
:0C648B001271DA80B3A24EB3925FA24EF1
:0164970022E2
:107582007A027BA37D02E4FF12642D502E9002A3A7
:10759200E07004A3E060249002A7E04480F07A0245
:1075A2007BA77D017F041258299002A7E0547FF047
:0C75B2007A027BA77D017F041258292279
:105E9700E49002A6F0A37450F0E4A3F0A374F8F022
:105EA700E4A3F0A3F0A37470F0A37401F0A3740348
:105EB700F0A374FFF0E4A3F03000199002A7E044C8
:105EC70008F09002ACE0FF9000BBE0540FFEEF4EED
:105ED7009002ACF030013E9002A7E04404F090023B
:105EE700ADE0FF9000BBE054F0FEEF4E9002ADF046
:105EF7009000BCE0FEA3E0FF7C007D3212252CE47D
:105F07007B257A01F9F8122304AD07AC06EC900261
:055F1700AEF0A3EFF065
:015F1C002262
:105E1000D24D9002C07403F09002C0E0FF14F0EF86
:105E200060727A027BA67D0B7F03125829505C902A
:105E300002BF7403F09002BFE0FFD3940B504E7A80
:105E4000027BBD7D0212642D9002BFE0FF7E007BCD
:105E50000124A3F9EE3402FA122189FD9002BDE07B
:105E6000B5051374A42FF9EE3402FA122189FF90BC
:105E700002BEE06F600C9002BFE064076004C24D98
:105E8000800B9002BFE02402F080AAC24D304D8802
:065E900080028084A24D97
:015E960022E9
:107545007A027BA37D02E4FF12642D502F9002A4E2
:10755500E0FF30E102D25CEF30E002D25E9002A3A0
:10756500E0FF30E307206B04D215D26DEF30E20265
:0D757500D2149002A4E030E203125E102256
:107B04007A027BBA7D027F0212642D500A9002BA77
:077B1400E09002A5F0F52648
:017B1B002247
:106634009002BC7403F09002BCE0FFD3940B505062
:106644007A027BBA7D0212642D9002BCE0FF7E00C8
:106654007B0124A3F9EE3402FA122189FD9002BAD7
:10666400E0B5051374A42FF9EE3402FA122189FF60
:106674009002BBE06F60109002BCE06407600812F7
:106684005E10400CD266229002BCE02402F080A688
:0166940022E3
:107941009002B07433F07A027BB07D017F0D125842
:107951002950129002A7E04420F07A027BA77D0112
:067961007F0412582922E8
:107B76009002A8E054FCF04FF07A027BA87D017FCA
:057B8600051258292240
:107BC7009002A7E04401F07A027BA77D017F0412AF
:037BD70058292208
:107BDA009002A7E054FEF07A027BA77D017F04128F
:037BEA00582922F5
:107BED009002A7E04402F07A027BA77D017F041288
:037BFD00582922E2
:107C00009002A7E054FDF07A027BA77D017F041269
:037C1000582922CE
:107506009002BCEEF0A3EFF09002BCE0FEA3E078A0
:1075160005CEC313CE13D8F99002AAF07A027BAA3D
:107526007D017F0712582950159002BCE0A3E09018
:0F75360002ABF07A027BAB7D017F08125829224D
:107C13009002A7E04410F07A027BA77D017F041253
:037C2300582922BB
:107C26009002A7E054EFF07A027BA77D017F041251
:037C3600582922A8
:107C39009002A9E044F8F07A027BA97D017F06123F
:037C490058292295
:107C4C009002A9E05407F07A027BA97D017F06120D
:037C5C0058292282
:107C5F009002A9E044E0F07A027BA97D017F061231
:037C6F005829226F
:107C72009002A9E0541FF07A027BA97D017F0612CF
:037C82005829225C
:107C85009002A9E04408F07A027BA97D017F0612E3
:037C950058292249
:107C98009002A9E054F7F07A027BA97D017F0612D1
:037CA80058292236
:107CBD009002A6E04FF07A027BA67D017F03125859
:027CCD0029226A
:107B1C009002A6E0FEEFF4FFEE5FF07A027BA67D0A
:077B2C00017F03125829221A
:1046590030610302479C30620302479C2003030236
:10466900479CE490053AF0A3F0C3900063E09512EB
:10467900900062E09511500330181ED3900065E058
:104689009512900064E09511400320180C20100940
:10469900201206201103301308C263E4900539F093
:1046A90022C39000A3E095129000A2E09511400367
:1046B900024795C3E5129510FFE511950FFED390BA
:1046C90000A5E09F9000A4E09E400302479590005A
:1046D900A6E0FEA3E0FFEE3395E0FDFC9002201278
:1046E9002437C31223B1500302479520630690056E
:1046F90039E004F09000A8E075F00AA4FF900539AC
:10470900E0C39FE5F06480F8748098500302479CE9
:10471900AD14E5142513FFE433FEEDC39FEE648069
:10472900F87480985063ED25E0240AF582E4340298
:10473900F583E0FEA3E0C39510FFEE950FFED3903D
:1047490000A5E09F9000A4E09E503BED25E0240ADF
:10475900F582E43402F583E0FEA3E0FF9000A2E0D5
:10476900FAA3E0FBC3EF9BEE9A401B74017E00A8FD
:1047790005088005C333CE33CED8F9FF90053AE05A
:104789004EF0A3E04FF00D8089D26322C263E4901A
:034799000539F0EF
:01479C0022FA
:1076DF00C24D30052D20162A306527C39002B4E025
:1076EF0094B49002B3E094005011D24D900538E05D
:1076FF0004F0C3940A400BD2168007C265E49005CC
:04770F0038F0A24D5F
:017713002253
:1054B200C3E5129510FFE511950FFEC3EF94B0EE10
:1054C2009404500AE5129464E51194055002D265E1
:1054D200900536E024FE605514605914606A146029
:1054E2007C2404600302556B20620330637B3064CA
:1054F2001590053AE05455FFA3E054559002BACFF7
:10550200F0A3EFF0801390053AE054AAFFA3E05411
:10551200AA9002BACFF0A3EFF09002BAE0FEA3E0A5
:10552200FF1275069005367402F0D261229005369C
:105532007403F0221276DF4030E4FFFE127506900B
:1055420005367404F0B264221276DF400790053605
:105552007405F0229005367401F0B264229005368B
:095562007401F0C262C263C2616F
:01556B00221D
:1079670030052220161F900537E004F0C3942D4000
:1079770014742DF020610EE4F0D26290053A74037E
:06798700F0A374FFF022E2
:0A7D05001246591279671254B22297
:10777E00FFD8FFE2FFECFFF60000000A001900231D
:10778E00002D00370041004B0055FFFBFFFCFFFDB5
:10779E00FFFEFFFFFFFF00000001000100020003DB
:0477AE0000040005CE
:04351E008F828E8387
:103522007E037FE8AD82AC8312252CC006C007AEB5
:1035320083AF82C3E49FFF74109EFEAB07FAE4F9E7
:10354200F8D007D0061223049002BD122484E47F2F
:103552000AFEFDFC9002BD122437D31223C7401D80
:103562009002BD12241EC3EF940AFFEE9400FEEDFA
:103572009400FDEC9400FC9002BD12248490479DBF
:10358200E493FE740193FFE4FCFD9002BD12243724
:10359200C31223C7400D9002BB7408F0A374B7F0A6
:1035A2000237059048DDE493FE740193FFE4FCFDCD
:1035B2009002BD122437D31223C7500D9002BB7460
:1035C2000EF0A374F7F002370590027CE09002BA85
:1035D200F075F00290479D1224DAE493FE74019391
:1035E200FFE4FCFD9002BD122437D31223C7403BF7
:1035F20090027CE0149002BAF09002BAE0FFC39409
:1036020000406975F002EF90479D1224DAE493FEC0
:10361200740193FFE4FCFD9002BD122437D3122300
:10362200C740499002BAE014F080CE90027CE004D8
:103632009002BAF09002BAE0FFC394A0502875F04D
:1036420002EF90479D1224DAE493FE740193FFE4A3
:10365200FCFD9002BD122437D31223C750089002FA
:10366200BAE004F080CE9002BAE014F09002BAE020
:1036720090027CF075F00290479D1224DAE493FEEA
:10368200740193FFE4FCFD9002BD12243712226BF9
:10369200E47B0AFAF9F8122279C004C005C006C018
:1036A200079002BAE0FF75F00290479F1224DAE415
:1036B20093FC740193FD75F002EF90479D1224DA9A
:1036C200C37401939DFFE4939CFEAB07FAE4F9F8FF
:1036D200D007D006D005D004122304AB07AA069067
:1036E200027CE024CEFFE434FFFE7C007D0A12213E
:1036F200E1EF2BFFEE3ACF24ABCF340A9002BBF0BE
:0B370200A3EFF09002BBE0FEA3E0FF8D
:01370D002299
:106FDC00D24D9002C3E514F0E5132514FFE433FE03
:106FEC009002C3E0C39FEE6480F87480985028E050
:106FFC00FF25E02485F582E43402AB82FAEF25E02C
:10700C00240EFF7D0212642D4005C24DA24D22902C
:09701C0002C3E004F080C1A24DA2
:017025002248
:10714A00D24D7A027B997D027F2212642D4002C2BF
:10715A004D7A027B9B7D027F2412642D4002C24D30
:10716A007A027B9D7D027F2612642D4002C24DE584
:10717A0013D39405400F7A027B9F7D027F28126405
:07718A002D4002C24DA24D91
:0171910022DB
:104C360012714A4003024D13900299E0FEA3E0FF71
:104C460012351E9000C6E02FFF9000C5E03EFEC262
:104C5600AC900224F0A3EFF0D2AC90029DE0FEA34C
:104C6600E0FF7C007D1112252CE47B0AFAF9F8128C
:104C76002304EF241FFFE43EFEC2AC900228F0A3FB
:104C8600EFF0D2ACE513D39405402A90029FE0FEE4
:104C9600A3E0FF7C007D1112252CE47B0AFAF9F8CB
:104CA600122304EF241FFFE43EFEC2AC90022AF05A
:104CB600A3EFF0D2AC900224E0FCA3E0FD90020248
:104CC600ECF0A3EDF0900204ECF0A3EDF0300D3D16
:104CD60090029BE0FEA3E0FF12351E9000C8E02F75
:104CE600FF9000C7E03EFEC2AC900226F0A3EFF0B4
:104CF600D2ACD3900203E09F900202E09E4006EE03
:0D4D0600F0A3EFF022900204EEF0A3EFF016
:014D1300227D
:1048DF009002BB1224A9000000009002BF1224A96D
:1048EF0000000000E4900200F0A3F09002B37417F0
:1048FF00F0A37470F0126FDC4003024A169002BAF4
:10490F00E514F0E5132514FFE433FE9002BAE0FD41
:10491F00C39FEE6480F874809840030249EDED2543
:10492F00E02485F582E43402F583E0FEA3E0FF7C0A
:10493F000E7DD812252CC006C0079000BFE0FEA345
:10494F00E0FFFBAA06E4F9F8D007D0061223049083
:10495F0002BF122484900200E0FEA3E0FFE4FCFDFE
:10496F009002BF122437D31223C7400E9002BF12FA
:10497F00241E900200EEF0A3EFF09002B3E0FEA32E
:10498F00E0FFE4FCFD9002BF122437C31223C7508F
:10499F000E9002BF12241E9002B3EEF0A3EFF02090
:1049AF006133C2AC9002BF12241E9002BAE025E020
:1049BF00240AF582E43402F583EEF0A3EFF0D2ACD3
:1049CF009002BB12241E9002BF12243712225E9057
:1049DF0002BB1224849002BAE004F0024912206153
:1049EF0026900200E0F511A3E0F5129002B3E0F576
:1049FF000FA3E0F510C2AC9002BB12241E90021E52
:074A0F00EEF0A3EFF0D2ACC2
:014A1600227D
:10561F00E49002BFF0A3F0A3F09002C1E0FFC394A7
:10562F000C40030256C9EF25E0247EF582E434775F
:10563F00F583E493FE740193FFFBAA06EA3395E02A
:10564F00F9F89002C1E025E02480F582E43477F583
:10565F0083E493FE740193FFEE3395E0FDFC122279
:10566F005EE47B02FAF9F8127380E47B0AFAF9F828
:10567F00122279EF24ABFBEE340AFAE43DF9E43C55
:10568F00F8900228E0FEA3E0FFE4FCFDC31223B173
:10569F00401F9002C1E025E02498F582E43477F5AD
:1056AF0083E493FF7401939002BFCFF0A3EFF080D8
:1056BF00099002C1E004F00256289002BFE0FEA359
:0256CF00E0FFFA
:0156D10022B6
:103E01009002BB1224A9000000007A027BA17D026E
:103E11007F2A12642D9002A1E0FEA3E0FFEE30E4C0
:103E21000944E09002A1F0A3EFF012561F9000C3E5
:103E3100E0FCA3E0FDC39002A2E09DFD9002A1E0A1
:103E41009CCD2FFFED3EFE3395E0FDFC7B187AFC07
:103E510079FF78FF122279C006C0079000C1E0FE09
:103E6100A3E0FFFBAA06EA3395E0F9F8D007D006F4
:103E710012738090027D12248490027D12241E9080
:103E810002B2E025E025E0243CF582E43402F5832A
:103E91001224849002B2E004F0C394104002E4F0D2
:103EA100E49002BAF09002BAE0FFC394105026A346
:103EB100122437EF25E025E0243CF582E43402F5B5
:103EC1008312241E12225E9002BB1224849002BA35
:103ED100E004F080D0E47B10FAF9F89002BB1224E0
:103EE1001E127380900281122484C22BC22A900078
:103EF10028E0FEA3E0FFC3E49FFFE49EFE3395E0CC
:103F0100FDFC900281122437C31223B15021900588
:103F1100F2E004F0C3940A4067740AF0D22BC2ACF9
:103F210090028112241E900220122484D2AC22908D
:103F31000028E0FEA3E0FFEE3395E0FDFC90028156
:103F4100122437D31223B140299005F1E004F094F3
:103F51000A402D740AF0D22A7D647FA07E0F126080
:103F61001FC2AC90028112241E900220122484D21E
:103F7100AC22C2AC9002201224A900000000D2ACF5
:013F8100221D
:107BA000127545C25E1248DF124C36305C05C25C6D
:047BB000123E01225E
:10635400E49002BAF0A3F0AF14E513FDE5142DFDAB
:10636400E433FCEFC39DEC6480F8748098501DEF17
:1063740025E02485F582E43402F583E0FCA3E0FD06
:106384009002BAEC8DF01222480F80CD9002BAE050
:10639400FEA3E0FF7C0E7DD812252CC006C007901A
:1063A40005DFE0FEA3E0FFFBAA06E4F9F8D007D07E
:0C63B400061223049000BFEEF0A3EFF0EF
:0163C00022BA
:1075F9009000C3E0FEA3E0FFC39002A2E09FFF90CA
:1076090002A1E09EFE3395E0FDFC7B187AFC79FF30
:1076190078FF1222799005D6122437127380EF4E23
:0A76290060089000C1EEF0A3EFF03E
:017633002234
:107CCF009002A1E0FFA3E09000C3CFF0A3EFF0225A
:1072B200900299E0FEA3E0FF12351EC39005DCE0C8
:1072C2009FFF9005DBE09EFE9000C5E0FCA3E0FD81
:1072D200C3EF9DFDEE9CFCC3ED9496EC648094801C
:1072E2005012ED946AEC6480947F40089000C5EEE1
:0472F200F0A3EFF026
:0172F6002275
:1072F70090029BE0FEA3E0FF12351EC39005DEE07F
:107307009FFF9005DDE09EFE9000C7E0FCA3E0FD37
:10731700C3EF9DFDEE9CFCC3ED9496EC64809480D6
:107327005012ED946AEC6480947F40089000C7EE99
:04733700F0A3EFF0E0
:01733B00222F
:10733C009005E1E0900497F09005E2E0900498F05D
:10734C009005E3E0900499F09005E4E090049AF045
:10735C009005E5E090049BF09005E6E090049CF02D
:10736C009005E7E090049DF07E047F97125A17D2A7
:04737C003AD23D22A2
:106C3900307C4BC27C9005DAE030E003126354905B
:106C490005DAE030E4031275F99005DAE030E5037E
:106C5900127CCF9005DAE030E2031272B29005DAC5
:106C6900E030E3031272F79005DAE030E7031273BC
:0F6C79003CE49005DAF0D2739005F57402F02236
:106DC400306D0DC26DD26BE49005F4F0127BED22B0
:106DD400306B3A127B04203134900087E075F00266
:106DE400A4FFAEF09005F4E004F0C39FEE6480F8D5
:106DF4007480984018C26BE4F0127C00307902C2AF
:0E6E040019C21BC21C301505C2151275822260
:1070B900306C0DC26CD26AE49005F3F0127BC722E2
:1070C900306A35127B0420302F900087E075F0027A
:1070D900A4FFAEF09005F3E004F0C39FEE6480F8DE
:1070E9007480984013C26AE4F0127BDA307807C2E0
:0970F90018C214127582C21A2299
:107A7700300719303B119003E7E004F0C394054049
:0D7A87000BD2397405F022E49003E7F022E1
:1066F6009002E4EEF0A3EFF0A3EDF0A3EAF0A3EB33
:01670600F0A2
:10670700C24D203941E4A3F09002E4E0FCA3E0FD90
:10671700A3E09002FAF0E4A3F09002E7E0FFA3E021
:106727009002FCCFF0A3EFF07B017FA0124512503F
:1067370004D24D80117F011271DA9002E9E004F072
:0D674700E0C3940540C2A24DB3923BA24DA9
:016754002222
:106755009002C6EEF0A3EFF0A3EDF0A3EAF0A3EBF1
:01676500F043
:10676600C24E203941E4A3F09002C6E0FCA3E0FD4E
:10677600A3E09002F0F0E4A3F09002C9E0FFA3E0EA
:106786009002F2CFF0A3EFF07B017FA0123A955072
:1067960004D24E80117F011271DA9002CBE004F030
:0D67A600E0C3940540C2A24EB3923BA24E48
:0167B30022C3
:1063C1007E027FBD7B08E4FD1278C9E49002BBF038
:1063D100A3F09002BBE0FEA3E0FFE4FCFD7BFF7AAB
:1063E10007F9F8D31223B1402E53B1F89002BBE064
:1063F100FEA3E07805C333CE33CED8F9241FFFE4E2
:106401003EFE7A027BBD7D011266F69002BBE47509
:10641100F00112224880BB7A027BBD7D087FE07EBD
:0B642100FF1266F6E49003E0F0A3F029
:01642C00224D
:1060A000C24D7A027BBA7D087FE07EFF126755926F
:1060B0004D9002BBE0FF9002BAE02F9002BCF0903E
:1060C00002BFE0FF9002BEE02F9002C0F09002BD40
:1060D000E0FF9002BCE0B507179002BAE0FEA3E033
:1060E0007C002400FFEC3E9003E0F0A3EFF0802A58
:1060F0009002C1E0FF9002C0E0B507179002BEE039
:10610000FEA3E07C002400FFEC3E9003E0F0A3EF50
:0C611000F08007E49003E0F0A3F0A24D43
:01611C002260
:106EF800E49002C4F07E047F971238D37E047F9713
:106F08007C027DBB7B071277B2E4FF74BB2FF5824E
:106F1800E43402F583E0FE9002C4E02EF00FEFB4F3
:106F280007E99002C4E09002C2F0A3745AF07A0212
:0B6F38007BBB7D097FF07EFF1266F638
:016F4300222B
:107406009003E0E0FCA3E0FDEC9002DCF0AF05A306
:10741600EFF09002DCE02F9002DFF09002DCE090CB
:1074260002E0F09002DDE09002E1F09002DFE090F1
:1074360002E3F07A027BDC7D087FE07EFF1266F6CF
:017446002223
:053C4E009002BBEFF045
:103C53006410701A7E037FE87C027DBC7B031277BD
:103C6300B27E037FEC7C027DBF1277B2801F7E049D
:103C73007F971238D37E047F977C027DBC7B03122F
:103C830077B27E047F9A7C027DBF1277B2900206E0
:103C9300E0FCA3E0FDEC9002C2F0A3EDF09002087B
:103CA300E0FCA3E0FDEC9002C4F0A3EDF090022C45
:103CB30012241E78181223D89002C6EFF090022C1B
:103CC30012241E78101223D89002C7EFF090022C12
:103CD30012241E78081223D89002C8EFF090022C09
:103CE30012241E9002C9EFF090023012241E78189D
:103CF3001223D89002CAEFF090023012241E7810DB
:103D03001223D89002CBEFF090023012241E7808D1
:103D13001223D89002CCEFF090023012241E9002AE
:103D2300CDEFF090021EE0FCA3E0FDAE047818CEC8
:103D3300C313CE13D8F99002CEF0EDAE047810CEB3
:103D4300C313CE13D8F99002CFF090021EE0FCA368
:103D5300E0FDEC9002D0F0A3EDF090022012241EBF
:103D630078181223EB9002D2EFF090022012241E57
:103D730078101223EB9002D3EFF090022012241E4E
:103D830078081223EB9002D4EFF090022012241E45
:103D93009002D5EFF0900224E0FCA3E0FDEC90024A
:103DA300D6F0A3EDF0900236E0FCA3E0FDEC900228
:103DB300D8F0A3EDF09002BBE09002DAF0A3745ABE
:103DC300F09003E0E0FEA3E0FF7A027BBC7D2012CB
:103DD30066F69003E0E475F0201222489003E0E0D9
:103DE300FEA3E0FFE4FCFD7BE07AFFF9F8D31223A6
:0D3DF300B15007E49003E0F0A3F012740655
:013E0000229F
:106498009003F2E02480FFE434FFEF7D00C454F061
:1064A800FC900401E02488FFE434FFFEEF7807C382
:1064B80033CE33CED8F92DFFEE3CFE900402E0FD3A
:1064C8007A047B031267557B017A047900900402F1
:1064D800E02403FD127ACE900402E02403F582E45E
:1064E8003404F583EFF0C29C9003FAE02400F582AF
:0A64F800E43404F583E0F599D2A026
:016502002276
:106207009003F2E02480FFE434FFEF7D00C454F0F4
:10621700FC9004A1E02488FFE434FFFEEF7807C375
:1062270033CE33CED8F92DFFEE3CFE9004A2E0FD2D
:106237007A047BA31267557B017A0479A09004A2A4
:10624700E02403FD127ACE9004A2E024A3F582E4B1
:106257003404F583EFF0758640C2A49003FBE02475
:0E626700A0F582E43404F583E0F5A1E4F586A9
:016275002206
:106276009003F2E02480FFE434FFEF7D00C454F085
:10628600FC900541E02488FFE434FFFEEF7807C365
:1062960033CE33CED8F92DFFEE3CFE900542E0FD1D
:1062A6007A057B431267557B017A05794090054252
:1062B600E02403FD127ACE900542E02443F582E401
:1062C6003405F583EFF0758640C2949003FCE02414
:0E62D60040F582E43405F583E0F591E4F586A9
:0162E4002297
:107192007E047F971238D37E047F977C047D037B25
:1071A200071277B27B017A047900900402E024038B
:1071B200FD127ACE900402E02403F582E43404F551
:1071C20083EFF0C29C9003FAE02400F582E43404D9
:0871D200F583E0F599D2A0223B
:106F44007E047F971238D37E047F977C047DA37BD5
:106F5400071277B27B017A0479A09004A2E024039B
:106F6400FD127ACE9004A2E024A3F582E43404F561
:106F740083EFF0758640C2A49003FBE024A0F58261
:0C6F8400E43404F583E0F5A1E4F5862276
:106F90007E047F971238D37E047F977C057D437BE8
:106FA000071277B27B017A057940900542E024030D
:106FB000FD127ACE900542E02443F582E43405F5D3
:106FC00083EFF0758640C2949003FCE02440F58284
:0C6FD000E43405F583E0F591E4F5862239
:1056D20020070302577D203A0302577DC23A303831
:1056E20005C2381263C19003E2E0FF7008A3E070C4
:1056F20004A3E06021EF6008E49003E2F0126498F2
:105702009003E3E06005E4F01262769003E4E06067
:1057120005E4F01262769003EFE0FF7008A3E070F8
:1057220004A3E06021EF6008E49003EFF0127192AD
:105732009003F0E06005E4F0126F449003F1E06042
:1057420005E4F0126F90303D05C23D126EF8303C18
:105752000CC23C9002BA7410F0FF123C4E30420C64
:10576200C2429002BA7401F0FF123C4E303F0CC2AA
:0B5772003F9002BA7402F0FF123C4EA0
:01577D002209
:104DEB00200703024EBD90002EE0FF9003DDE00490
:104DFB00F0C39F4009E4F07E047F971238D39003F1
:104E0B00DEE475F001122248FEC3E5F09410EE9437
:104E1B000E400BE49003DEF0A3F0D23AD23D202AF1
:104E2B001ED241304006C240D23AD24230190B302A
:104E3B003E08C23ED23AD23F8005201902D23E3004
:104E4B00416990002CE0FEA3E0FFEE3395E0FDFC02
:104E5B00900220122437C31223B1404F9003E5E098
:104E6B007002A3E070147E047F971238D37E047F08
:104E7B00977C037DE87B071277B290002BE0FF7ED7
:104E8B00007C007D3C1221E19003E5E475F00112FA
:104E9B002248FCD3E5F09FEC9E4017E49003E5F02D
:104EAB00A3F0D240C241D23AD23C22E49003E5F0C7
:034EBB00A3F0223F
:031053000262E551
:1062E500C0E0C083C082C0D075D000C007C086752D
:1062F500860030D807C2D87F0112102E30D907C2C8
:10630500D97F0212102E30DA07C2DA7F0412102E5E
:1063150030DB07C2DB7F0812102E30DC07C2DC7FC2
:106325001012102E30DD07C2DD7F2012102E30DE58
:1063350007C2DE7F4012102E30DF07C2DF7F8012DA
:0F634500102ED086D007D0D0D082D083D0E032B7
:03102B00021003AD
:10100300C0E0C083C082C0D0C086758640C28F75E1
:1010130086001279B3D086D0D0D082D083D0E0328C
:1058D400307D0302597575090F20A70575090180EC
:1058E4000620B003750902E509650C6038050EE56C
:1058F4000E7002050DC3E50B940AE50A9400406599
:10590400E50E940AE50D94004067E50B9490E50AD2
:1059140094014008E50C4440F5088003850C08D246
:105924007D80428040E509640F6037E4F50DF50E93
:10593400050BE50B7002050AB4900EE50AB40109E3
:10594400E50C4410F508D27D22E50BB4B023E50A3A
:10595400B4041E750A01750B90E50C4420F508D2B9
:105964007D2275080FE4F50AF50BF50DF50E850992
:015974000C26
:01597500220F
:10771400AB07AA06C2AF43A701EAF5F7AF038FFB95
:10772400AF058FFC75F26E75F30575F40A75F509EE
:10773400EAADF7B50509E475F6060000000000534C
:05774400A7FED2AF22F8
:10798D00D250E4FDFCEF2DFBEE3C8B82F583E493AE
:10799D006004C250800D0DBD00010CE4B505E6EC90
:0579AD00B402E2A2504B
:0179B20022B2
:086982009002C0EEF0A3EFF05B
:10698A00D250AE04AF05E4A3F0A3F09002C2E0FC3B
:10699A00A3E0FDC3EC940250369002C1E02DFD90B5
:1069AA0002C0E03C8D82F583E493FD9002C2E0FAD6
:1069BA00A3E02FF582EE3AF583E0FCED6C6004C2A9
:1069CA0050800C9002C2E475F00112224880BCA2E9
:0169DA00506C
:0169DB002299
:085CFC009002C0EEF0A3EFF0EE
:105D0400C250AF05A3ECF0A3EFF0E4FDFC9002C099
:105D1400E0FAA3E0FB2DF5FBEB2DEA3CF5F7A3E05D
:105D2400FEA3E02DF582EE3CF583E0F5FC75F26E02
:105D340020AF3D75F305E5A7603275F40A9005F6CA
:105D4400E06455702375F5099002C1E02D9002C0FE
:105D5400E03CABF7B5030DE475F606000000000067
:105D6400D2508010C2508019C2508015C250801188
:105D7400C250800D0DBD00010CED7003EC64027087
:035D84008CA2509E
:015D870022F9
:0E5B4A009002BCEEF0A3EFF0A3ECF0A3EDF0A0
:105B5800C24F53B1F8C2AF43A7019002BCE0FF7E29
:105B680000F5F775F2E620AF5B75F305E5A760541D
:105B780075F40A9005F6E06455704975F509ADF7B6
:105B8800EF6D7001EE703D75F606000000000090A4
:105B980002BCE0FEA3E0FF12798D50289002BCE021
:105BA800FEA3E0FFA3E0FCA3E0FD125CFC5015900F
:105BB80002BCE0FEA3E0FFA3E0FCA3E0FD126982C3
:105BC8005002D24FE4F5F2F5F3F5F4F5F5F5F65396
:085BD800A7FEF5F7D2AFA24FC2
:015BE00022A2
:10504500C24DC24E207203025105C2729005F6741C
:1050550055F0E513D39405400C9002BA7427F0A3DC
:105065007410F0800A9002BA7413F0A37488F0905B
:1050750002BAE0FEA3E0FFC390021FE09F90021E6C
:10508500E09E406B9001FEE0645A7004A3E064A5C5
:10509500705DFDFCFFFE125B4A4023E4FDFCFFFE54
:1050A500125B4A4019D24D74FF9001FEF0A3F0FD4A
:1050B5007FFE7E011277147DFF7FFF127714E4FDDA
:1050C500FCFF7E02125B4A402AE4FDFCFF7E0212D1
:1050D5005B4A401FD24E74FF9001FEF0A3F0FD7FA6
:1050E500FE7E031277147DFF7FFF1277148004D2B2
:1050F5004DD24EE49005F6F0304D05304E02D2719A
:015105002287
:0E67B4009002BAEEF0A3EFF0A3EAF0A3EBF030
:1067C200D24DAE04AF058E158F16C2AF43A701534B
:1067D200B1F8E4FFFED39002BDE09F9002BCE09EC0
:1067E20040279002BBE02FFD9002BAE03E8D82F579
:1067F20083E493851682851583F00516E5167002EB
:1068020005150FBF00010E80CC53A7FED2AFA24DDB
:016812002263
:107B8B003073119005F5E004F0C394024006C27304
:057B9B00E4F0D27222AB
:1078F300C24D43A701EEC313FEEF1325E0FFEE33A2
:107903008F82F583740193B4A507E493B45A02D22A
:067913004D53A7FEA24D3A
:01791900224B
:057815009002BAEFF043
:10781A00758640758830AE04AF057C1F7D40122501
:10782A002CE4FB7A01F9F8122304C3E49FFFE49ED7
:0A783A00FE8F8CF58DD28AE4F586EE
:017844002221
:0579D7009002BAEFF080
:1079DC00A2AFE433FFC2AF43B208000000000000C6
:0C79EC00000053B26043B20424FF92AFCD
:0179F800226C
:105F1D009005EBEEF0A3EFF0A3EDF075C7B0900593
:105F2D00EBE0FEA3E0FFFBAA06E4F9F87FD87EB80C
:105F3D007D05FC1273808FCC9005EBE0FEA3E0FF96
:105F4D00FBAA06E4F9F87FD87EB87D05FC127380B4
:105F5D0078081223EB8FCDAFCDEFFEADCC7C00E4F6
:105F6D002DFFEC3EFE9005EDE0FBFD1221E17D6481
:105F7D001221F38FCEAFCDEFFEADCC7C00E42DFF23
:105F8D00EC3EFEAD031221E17D641221F3EEF5CF5F
:015F9D0022E1
:105F9E009005EEEEF0A3EFF0A3EDF075B6B0900520
:105FAE00EEE0FEA3E0FFFBAA06E4F9F87FD87EB888
:105FBE007D05FC1273808FAE9005EEE0FEA3E0FF30
:105FCE00FBAA06E4F9F87FD87EB87D05FC12738033
:105FDE0078081223EB8FAFAFAFEFFEADAE7C00E4CF
:105FEE002DFFEC3EFE9005F0E0FBFD1221E17D64FD
:105FFE001221F38FA4AFAFEFFEADAE7C00E42DFF08
:10600E00EC3EFEAD031221E17D641221F3EEF5A507
:01601E00225F
:10601F009002BFEEF0A3EFF0A3EDF075B7B09002D2
:10602F00BFE0FEA3E0FFFBAA06E4F9F87FD87EB835
:10603F007D05FC1273808FBC9002BFE0FEA3E0FFD2
:10604F00FBAA06E4F9F87FD87EB87D05FC127380B1
:10605F0078081223EB8FBDAFBDEFFEADBC7C00E423
:10606F002DFFEC3EFE9002C1E0FBFD1221E17D64AD
:10607F001221F38FBEAFBDEFFEADBC7C00E42DFF50
:10608F00EC3EFEAD031221E17D641221F3EEF5BF6C
:01609F0022DE
:1071DA00E5B2547070067C067D868020E5B2547054
:1071EA00FEBE20067C037D438012E5B25470FEBECB
:1071FA0040067C017DA180047C007D8BE4FEEEC309
:10720A009F5014E4FBFAC3EB9DEA9C50070BBB00AA
:07721A00010A80F20E80E77B
:01722100224A
:1065690090002FE0645A705A900061E0645A7052AA
:10657900900073E0645A704A900088E0645A70424F
:1065890090008DE0645A703A900098E0645A703235
:106599009000A1E0645A702A9000A9E0B45A2390AF
:1065A90000BAE0B45A1C9000BEE0B45A159000CA73
:1065B900E0B45A0E9001FEE0645A7004A3E064A5A9
:0665C9006002C322D32290
:0878C9009002C6EEF0A3EFF0FF
:1078D100E4FFEFC39B501A9002C6E0F8A3E0F582E3
:1078E1008883EDF09002C6E475F0011222480F8002
:0178F100E1B5
:0178F2002273
:0877B2009002DCEEF0A3EFF001
:1077BA00E4FFEFC39B50239002DCE0F8A3E0F582DC
:1077CA008883E08D828C83F00DBD00010C9002DC71
:0A77DA00E475F0011222480F80D878
:0177E4002282
:0C7CED00758E5543870100000000002246
:0C7CF900758E5543870200000000002239
:107872009005EAE064127023204306204403304559
:107882001A207317207214C2AFE4F5A8F5A9F5887F
:0C789200F5E8F59DF59CF5981200002229
:10702600D228D229201403301602C22820110F209C
:10703600130C201B09201C06201503301602C2293A
:10704600202B0E201009201206201803301A02C227
:1070560028202A05301902C229201B06201C0330CD
:0A7066001502C228301A02C22922C6
:10784500127026A276302801B34008A277302901AC
:10785500B35019A2289276A2299277A229E433FF80
:0D78650025E0FFA228E4334FFF127B7622BE
:10722200201844C3900063E09512900062E095112B
:10723200501F9003BFE475F001122248FEC3E5F02F
:107242009401EE94004020D218E49003BFF0A3F022
:1072520022D3900065E09512900064E095114007FA
:08726200E49003BFF0A3F02249
:10726A00201944D3900075E09510900074E0950FB2
:10727A00401F9003C1E475F001122248FEC3E5F0F5
:10728A009401EE94004020D219E49003C1F0A3F0D7
:10729A0022C3900077E09510900076E0950F500792
:0872AA00E49003C1F0A3F022FF
:106C880020104B90008EE0FEA3E0FF900204E0FC91
:106C9800A3E0FDD39FEC9E401F9003D1E475F00163
:106CA800122248FEC3E5F09401EE94004020D21071
:106CB800E49003D1F0A3F022900090E0FEA3E0FF5F
:0F6CC800C3ED9FEC9E5007E49003D1F0A3F022A0
:106CD70020124B900092E0FEA3E0FF900202E0FC3E
:106CE700A3E0FDC39FEC9E501F9003D5E475F00110
:106CF700122248FEC3E5F09401EE94004020D21220
:106D0700E49003D5F0A3F022900094E0FEA3E0FF07
:0F6D1700D3ED9FEC9E4007E49003D5F0A3F0224C
:106D260020114B900099E0FEA3E0FF900204E0FCE6
:106D3600A3E0FDD39FEC9E401F9003D3E475F001C2
:106D4600122248FEC3E5F09401EE94004020D211D1
:106D5600E49003D3F0A3F02290009BE0FEA3E0FFB3
:0F6D6600C3ED9FEC9E5007E49003D3F0A3F022FF
:106D750020134B90009DE0FEA3E0FF900202E0FC93
:106D8500A3E0FDC39FEC9E501F9003D7E475F0016F
:106D9500122248FEC3E5F09401EE94004020D21380
:106DA500E49003D7F0A3F02290009FE0FEA3E0FF5C
:0F6DB500D3ED9FEC9E4007E49003D7F0A3F022AC
:10763400307E371248DF124C3612722212726A12EE
:107644006C88126CD7126D26126D7590053FE0049C
:10765400F0C394024014C27E205D09203906207BC9
:0B76640003307103D2662212425A224A
:104EBE0020185C201459C3900063E0951290006294
:104ECE00E095115033900066E075F00AA4FFAEF045
:104EDE009003BFE475F001122248FCC3E5F09FEC8D
:104EEE009E5003024F81D218C278E49003BFF0A304
:104EFE00F09003D9F0A3F022D3900065E0951290C4
:104F0E000064E09511406CE49003BFF0A3F0222002
:104F1E007861D3900065E09512900064E0951140A1
:104F2E003C900067E075F00AA4FFAEF09003D9E460
:104F3E0075F001122248FCC3E5F09FEC9E40343020
:104F4E000E06D278D26C8007C218C214127582E493
:104F5E009003BFF0A3F09003D9F0A3F022C390000A
:104F6E0063E09512900062E095115007E49003D92A
:044F7E00F0A3F0228A
:10510600201959D3900075E09510900074E0950F22
:105116004033900078E075F00AA4FFAEF09003C12A
:10512600E475F001122248FCC3E5F09FEC9E5003A3
:105136000251C1D219C279E49003C1F0A3F09003E1
:10514600DBF0A3F022C3900077E09510900076E0A4
:10515600950F5067E49003C1F0A3F02220795CC359
:10516600900077E09510900076E0950F503790000C
:1051760079E075F00AA4FFAEF09003DBE475F00168
:10518600122248FCC3E5F09FEC9E402F300F06D25A
:1051960079D26D8002C219E49003C1F0A3F09003A6
:1051A600DBF0A3F022D3900075E09510900074E038
:0C51B600950F4007E49003DBF0A3F0220B
:1051C20020105E90008EE0FEA3E0FF900204E0FC5F
:1051D200A3E0FDD39FEC9E4031900096E075F01461
:1051E200A4FFAEF09003D1E475F001122248FAC395
:1051F200E5F09FEA9E500302527DD210E49003D163
:10520200F0A3F09003C3F0A3F022900090E0FEA37D
:10521200E0FFC3ED9FEC9E5062E49003D1F0A3F057
:1052220022900090E0FEA3E0FF900204E0FCA3E0E5
:10523200FDC39FEC9E502E900096E075F014A4FFE3
:10524200AEF09003C3E475F001122248FAC3E5F010
:105252009FEA9E4026C210E49003D1F0A3F090038F
:10526200C3F0A3F02290008EE0FEA3E0FFD3ED9FF7
:0C527200EC9E4007E49003C3F0A3F02280
:10527E0020125E900092E0FEA3E0FF900202E0FC9E
:10528E00A3E0FDC39FEC9E5031900096E075F014A4
:10529E00A4FFAEF09003D5E475F001122248FAC3D4
:1052AE00E5F09FEA9E5003025339D212E49003D5E3
:1052BE00F0A3F09003C7F0A3F022900094E0FEA3B9
:1052CE00E0FFD3ED9FEC9E4062E49003D5F0A3F097
:1052DE0022900094E0FEA3E0FF900202E0FCA3E027
:1052EE00FDD39FEC9E402E900096E075F014A4FF27
:1052FE00AEF09003C7E475F001122248FAC3E5F050
:10530E009FEA9E4026C212E49003D5F0A3F09003CC
:10531E00C7F0A3F022900092E0FEA3E0FFC3ED9F42
:0C532E00EC9E5007E49003C7F0A3F022AF
:10533A0020115E900099E0FEA3E0FF900204E0FCD9
:10534A00A3E0FDD39FEC9E4031900096E075F014E7
:10535A00A4FFAEF09003D3E475F001122248FAC319
:10536A00E5F09FEA9E50030253F5D211E49003D36D
:10537A00F0A3F09003C5F0A3F02290009BE0FEA3F7
:10538A00E0FFC3ED9FEC9E5062E49003D3F0A3F0DC
:10539A002290009BE0FEA3E0FF900204E0FCA3E061
:1053AA00FDC39FEC9E502E900096E075F014A4FF6A
:1053BA00AEF09003C5E475F001122248FAC3E5F095
:1053CA009FEA9E4026C211E49003D3F0A3F0900313
:1053DA00C5F0A3F022900099E0FEA3E0FFD3ED9F71
:0C53EA00EC9E4007E49003C5F0A3F02205
:1053F60020135E90009DE0FEA3E0FF900202E0FC19
:10540600A3E0FDC39FEC9E5031900096E075F0142A
:10541600A4FFAEF09003D7E475F001122248FAC358
:10542600E5F09FEA9E50030254B1D213E49003D7ED
:10543600F0A3F09003C9F0A3F02290009FE0FEA332
:10544600E0FFD3ED9FEC9E4062E49003D7F0A3F01B
:105456002290009FE0FEA3E0FF900202E0FCA3E0A2
:10546600FDD39FEC9E402E900096E075F014A4FFAD
:10547600AEF09003C9E475F001122248FAC3E5F0D4
:105486009FEA9E4026C213E49003D7F0A3F0900350
:10549600C9F0A3F02290009DE0FEA3E0FFC3ED9FBC
:0C54A600EC9E5007E49003C9F0A3F02234
:1069DC00201A5590006D12241E90027D122437D37C
:1069EC001223B1402A900071E075F00AA4FFAEF0BA
:1069FC009003CDE475F001122248FCC3E5F09FEC46
:106A0C009E4025D21AD26CE49003CDF0A3F0222044
:106A1C006A16D39003CEE094009003CDE09400402E
:096A2C000774FFF5F01222482264
:106A3500201B5590007D12241E90027D122437C321
:106A45001223B1502A900081E075F00AA4FFAEF040
:106A55009003BBE475F001122248FCC3E5F09FECFE
:106A65009E4025E49003BBF0A3F0D21BD26D2220FB
:106A75006B16D39003BCE094009003BBE0940040F8
:096A85000774FFF5F0122248220B
:106A8E00201C5590008212241E90027D122437C3C2
:106A9E001223B1502A900086E075F002A4FFAEF0EA
:106AAE009003BDE475F001122248FCD3E5F09FEC93
:106ABE009E4025E49003BDF0A3F0D21CD26D22209F
:106ACE006B16D39003BEE094009003BDE09400409B
:096ADE000774FFF5F012224822B2
:107A3A00207E1B124EBE1251061251C212527E12E3
:0F7A4A00533A1253F61269DC126A35126A8E2211
:10611D00300272201B06201C03301539900072E0EE
:10612D0075F014A4FFAEF09003CFE475F0011222C8
:10613D0048FCC3E5F09FEC9E401BE49005F4F09005
:10614D0003CFF0A3F0C21BC21CC26DC26B3015058C
:10615D00C215127582301A2D900072E075F014A4DC
:10616D00FFAEF09003CBE475F001122248FCD3E5AD
:10617D00F09FEC9E400FE49003CBF0A3F0C21A9079
:06618D0005F3F0C26A22D6
:107A9400300719307A11900496E004F0C39405403D
:0D7AA4000BD27B7405F022E4900496F022D2
:0E68CC009002F1EFF0A3EDF0A3EAF0A3EBF0E1
:1068DA00C250207B40E4A3F09002F1E0FD7C00A3CB
:1068EA00E09002FAF0E4A3F09002F3E0FFA3E09054
:1068FA0002FCCFF0A3EFF0E4FB7FDE124512500456
:10690A00D25080117F011271DA9002F5E004F0E0B2
:0C691A00C3940540C3A250B3927AA2506F
:01692600224E
:0E6927009002E7EFF0A3EDF0A3EAF0A3EBF08F
:10693500C24F207B40E4A3F09002E7E0FD7C00A37A
:10694500E09002F0F0E4A3F09002E9E0FFA3E0900C
:1069550002F2CFF0A3EFF0E4FB7FDE123A9550048C
:10696500D24F80117F011271DA9002EBE004F0E062
:0C697500C3940540C3A24FB3927AA24F16
:0169810022F3
:0838D3009002DCEEF0A3EFF01F
:1038DB00C24E7A027BDE7D09E4FF126927400302A8
:1038EB003A929002E5E030E003023A859002E0E084
:1038FB0020E7030239A49002DEE0FF54709450409D
:10390B00030239A4EF540F940940030239A4E05485
:10391B007F945940030239A4A3E0FF547094505094
:10392B0078EF540F94095071E0547F9459506AA367
:10393B00E0FF543094205061EF540F9409505AE03B
:10394B00542F94245053A3E0FF54309430504AEF3B
:10395B00540F94095043E0543FFF9431503BEF60B8
:10396B0038A3E0FF54109410502FEF540F940950CC
:10397B0028E0541FFF94125020EF601DA3E0FF546A
:10398B00F094905014EF540F9409500DE09499500B
:10399B0008A3E05407940640779002DCE0FEA3E016
:1039AB00FFF5828E83E09002DEF08F828E83A3E0A0
:1039BB009002DFF09002DCE0A3E0F5828E83A3A3FC
:1039CB00E09002E0F08F828E83A3A3A3E09002E14C
:1039DB00F09002DCE0A3E02404F582E43EF583E002
:1039EB009002E2F0EF2405F582E43EF583E09002CD
:1039FB00E3F09002DCE0A3E02406F582E43EF583DD
:103A0B00E09002E4F07E027FDE125A17924E80772E
:103A1B009002DEE0FF9002DCE0FCA3E0FDF5828C7F
:103A2B0083EFF09002DFE08D828C83A3F09002E0B5
:103A3B00E0541F8D828C83A3A3F09002E1E08D8272
:103A4B008C83A3A3A3F09002E2E0FFED2404F582A4
:103A5B00E43CF583EFF09002E3E0FFED2405F58203
:103A6B00E43CF583EFF09002E4E0FFED2406F582F1
:103A7B00E43CF583EFF0D24E800D9002DCE0FEA328
:093A8B00E0FF125A17924EA24E00
:013A9400220F
:085A17009002E7EEF0A3EFF0AE
:105A1F00C24FA37490F07A027BE97D017F07126871
:105A2F00CC924F9002E7E0FEA3E0FFF5828E83E079
:105A3F009002EAF08F828E83A3E09002EBF0900247
:105A4F00E7E0FCA3E0FDF5828C83A3A3E044809004
:105A5F0002ECF08D828C83A3A3A3E09002EDF09073
:105A6F0002E7E0A3E0FF2404F582E43EF583E09033
:105A7F0002EEF0EF2405F582E43EF583E09002EFAD
:105A8F00F09002E7E0A3E02406F582E43EF583E020
:105A9F009002F0F07A027BEA7D07E4FF1268CC9265
:035AAF004FA24FB4
:015AB20022D1
:085C6F009002BAEEF0A3EFF081
:105C7700C24DE49002C5F07E027FBC7B09FD12781D
:105C8700C97A027BBC7D097FF07EFF126755E4FF6E
:105C970074BC2FF582E43402F583E0FE9002C5E080
:105CA7002EF00FEFB407E99002C5E0FF9002C3E0C2
:105CB700B50706A3E0645A601BE49002BCF0A3F0AA
:105CC700A37412F0A37401F0A37405F0A37420F079
:105CD700A37405F07E027FBC9002BAE0FCA3E0FD4E
:105CE7007B071277B29002BAE0FEA3E0FF1238D327
:045CF700924DA24DDB
:015CFB002286
:104B360000070E091C1B1215383F363124232A2D77
:104B460070777E796C6B6265484F464154535A5D67
:104B5600E0E7EEE9FCFBF2F5D8DFD6D1C4C3CACD57
:104B660090979E998C8B8285A8AFA6A1B4B3BABD47
:104B7600C7C0C9CEDBDCD5D2FFF8F1F6E3E4EDEA37
:104B8600B7B0B9BEABACA5A28F88818693949D9A27
:104B96002720292E3B3C35321F18111603040D0A17
:104BA6005750595E4B4C45426F68616673747D7A07
:104BB600898E878095929B9CB1B6BFB8ADAAA3A4F7
:104BC600F9FEF7F0E5E2EBECC1C6CFC8DDDAD3D4E7
:104BD600696E676075727B7C51565F584D4A4344D7
:104BE600191E171005020B0C21262F283D3A3334C7
:104BF6004E49404752555C5B7671787F6A6D6463B7
:104C06003E39303722252C2B0601080F1A1D1413A6
:104C1600AEA9A0A7B2B5BCBB9691989F8A8D848396
:104C2600DED9D0D7C2C5CCCBE6E1E8EFFAFDF4F386
:107ACE00E4FFEDD3940040131221896F904B36934F
:0B7ADE00FF740129F9E43AFA1D80E76B
:017AE900227A
:10791A00D2527D807CBBE5C820E31053B1F8ED4C10
:10792A006009ED1D70011C80ED80EBE5D154F86F04
:06793A006002C252A252DD
:017940002224
:104512009002F9EBF09002F6EFF0A3ECF0A3EDF0CD
:10452200D25190030274BBF0A37480F09002FEEFAC
:10453200F0A3EDF09002FCE0FEA3E0F5828E83E0B2
:10454200900300F07B017A0279FE7D03127ACE900D
:104552000301EFF09002FAE0D394005003024656B2
:1045620043E6C043D10143C80175C8607F08127990
:104572001A400C7F1012791A4005C251024633903C
:1045820002F6E0F58D75C8407F1812791A4005C20F
:10459200510246339002F9E0B401159002F7E0F5BA
:1045A2008D75C8407F2812791A4005C251024633E0
:1045B2009002F7E0A3E0F58D75C8407F2812791AC2
:1045C2004004C251806B9002FBE06401702EA3E0B4
:1045D200FEA3E0F5828E83E0F58D75C8407F281238
:1045E200791A4004C2518049900301E0F58D75C8E3
:1045F200407F2812791A4039C2518035E4FE900278
:10460200FAE0FFEEC39F50299002FCE0FCA3E0F524
:10461200828C83E0F58D75C8407F2812791A400498
:10462200C251800D9002FCE475F0011222480E8006
:10463200CD75C850E5C830E41B53B1F8900302E0D1
:104642007002A3E0600E90030274FFF5F01222489C
:0646520080E280E0A251AD
:01465800223F
:0A3A9500AA079002EDECF0A3EDF09B
:103A9F00D250E4900323F0A374BBF0A37480F09092
:103AAF0002F5EAF0A3EDF0EA4401A3F09002F0E092
:103ABF00D394005003023C4B43E6C043D10143C8AB
:103ACF000175C8607F0812791A400C7F1012791A9D
:103ADF004005C250023C288A8D75C8407F18127964
:103AEF001A4005C250023C28EBB401159002EDE0DC
:103AFF00F58D75C8407F2812791A4005C250023CD7
:103B0F00289002EDE0A3E0F58D75C8407F2812796B
:103B1F001A4005C250023C2875C8607F0812791AF6
:103B2F00400C7F1012791A4005C250023C28EA441B
:103B3F0001F58D75C8407F4012791A4005C25002B9
:103B4F003C28E49002F4F09002F0E0FF9002F4E0E1
:103B5F00FEC39F50579002F1E07031EF14B5060A83
:103B6F0075C8407F5812791A800875C8447F501263
:103B7F00791A9002F2E0FEA3E0F5828E83E58DF0D4
:103B8F009002F2E475F001122248801875C8447F44
:103B9F005012791A9002F4E024F8F582E43402F519
:103BAF0083E58DF09002F4E004F0809B9002F1E049
:103BBF006401706575C8407F5812791A900323E528
:103BCF008DF07B017A0279F59002F0E02403FD126B
:103BDF007ACE900323E0B5073EE49002F4F0900212
:103BEF00F0E0FF9002F4E0FEC39F502D74F82EF525
:103BFF0082E43402F583E0FF9002F2E0FCA3E0F5EB
:103C0F00828C83EFF09002F2E475F001122248905B
:103C1F0002F4E004F080C7C25075C850E5C830E424
:103C2F001B53B1F8900324E07002A3E0600E9003E1
:0E3C3F002474FFF5F012224880E280E0A250CB
:013C4D002254
:107B330075C632E4F5E6F5D1758A2075D10275C8AC
:077B4300407589FFF58D225A
:0366950075C43297
:10669800E4F5877598509002BA747FF0A374CCF033
:1066A8009002BAE0F59D759CCCE0FEA3E0FFFBE408
:1066B800C39BFF74809EFEE49400FDE49400FCE418
:1066C8007B10FAF9F8122279EC121D72A804A905B8
:1066D800AA06AB077F557E557D507C44121C7D125F
:0D66E8001DB08F9E439D80759A0A759BFF23
:0166F5002282
:03102300026B97C6
:106B9700C0E0C0F0C083C082C0D075D000C000C0C4
:0D6BA70001C002C003C004C005C006C00745
:106BB400C086758600309807C298AF99125AB330D0
:096BC4009905C29912556CD086A6
:106BCD00D007D006D005D004D003D002D001D0001C
:0B6BDD00D0D0D082D083D0F0D0E032C6
:10479D0080B678FA71C46B0C64C760C25B2755EBA9
:1047AD0051074C7449A2458441AA3E0D3AAB384A93
:1047BD00354132682FBB2D382B7A29362715251414
:1047CD00233121C320101E761CF41B881A79192F52
:1047DD0017F816D215BC14DD13E212F41213113EA4
:1047ED0010970FD50F1E0E700DCC0D3E0CA90C1B86
:1047FD000B940B140AA80A3309C5095B08F7089D29
:10480D00084207EB0798074A070406BC06770636E9
:10481D0005F705BD0584054D051904E804B9048B9C
:10482D0004600436040E03E803C303A0037E035E95
:10483D00033F0321030402E902CF02B6029E028662
:10484D000270025B02470232021F020D01FC01EBF6
:10485D0001DA01CB01BC01AE01A001920185017904
:10486D00016D01620156014B01410137012E0124F9
:10487D00011B0113010B010300FB00F300EC00E52C
:10488D0000DF00D800D200CC00C600C000BA00B5D1
:10489D0000B000AB00A700A2009D0099009500910B
:1048AD00008D008900850082007F007B00780075F7
:1048BD000072006F006C0069006600640061005FAB
:1048CD00005C005A0058005600530051004F004E36
:0248DD00004C8D
:03100000027A1A57
:107A1A0075819F007808760008B8A0FAE490000003
:107A2A00F0A3A882A983B8DCF7B907F400025D883D
:10370E00A2AF924DC2AF900234E0FFA3E090032827
:10371E00CFF0A3EFF090022C12241E900346122439
:10372E008490023012241E90037912248490023663
:10373E00E0FFA3E0900367CFF0A3EFF0900220121A
:10374E00241E90037E122484900224E0FFA3E090B6
:10375E000377CFF0A3EFF090021EE0FEA3E0FFE4AC
:10376E00FCFD90035012248485111C85121D850FBB
:10377E001A85101B9003621224A900000000E49029
:10378E000375F0A3F0A24D92AF90034F741EF0900C
:10379E00036E745AF0A3740BF0A3740FF0900369C8
:1037AE001224A9FFFF7748E490036DF09003720492
:1037BE00F090038A7414F090033F743EF0A374806B
:1037CE00F0A3E4F0A37411F09003737406F0A374E5
:1037DE0022F090038C743CF0900003E02438FE90AD
:1037EE000002E034FF900326F0A3CEF090035A744B
:1037FE000FF0900361740AF0900014E0FFA3E090C4
:10380E000382CFF0A3EFF090034E745AF0E513FB52
:10381E007A007C117D94FF7E001221E1E4FCFD9084
:10382E0003301224847C0B7DB8AF037E001221E19D
:10383E00E4FCFD900356122484900366743CF090D1
:10384E00038B7414F0900334740FF090037D741492
:10385E00F0900371740AF090032A1224A90000005C
:10386E0028900345741EF0900343740BF0A374412B
:10387E00F0900354740BF0A37441F0900384E4F0C1
:10388E00A37432F090034AE4F0A37405F090033B66
:10389E00E4F0A37469F0900386E4F0A37464F090EE
:1038AE00034CE4F0A3741EF090033DE4F0A37462A5
:1038BE00F09003887401F0A37490F090035FE4F02D
:0438CE00A3744BF0A4
:0138D20022D3
:106BE800A2AF924DC2AF900328E0FFA3E090023419
:106BF800CFF0A3EFF090034612241E90022C12242B
:106C08008490037912241E90023012248490036722
:106C1800E0FFA3E0900236CFF0A3EFF0A25A922251
:106C2800A25B92209000B9E024FF9221A24D92AF7E
:016C38002239
:067D0F005AA569963CC371
:104A17007F647E00E49002BCF09002BCE0FDC3948A
:104A27000A4003024B35ED25E02402F582E4340009
:104A3700F583E0FCA3E0D3951DEC951C5003024BD6
:104A47002C9002BCE0705790007AE0FCA3E0FDD305
:104A5700951DEC951C5003301906E4FEFF024B35FB
:104A6700C3E51D9DFFE51C9CFE7C007D0A12252CDD
:104A7700EEC0E0EFC0E090007AE0FEA3E0FFC39055
:104A87000003E09FFF900002E09EFECBEFCBFAE42D
:104A9700F9F8D0E0FFD0E0FE122304024B35900274
:104AA700BCE025E02400F582E43400F583E0FEA3B2
:104AB700E0FFC3E51D9FFFE51C9EFE7C007D0A12FB
:104AC700252CECC0E0EDC0E0EEC0E0EFC0E09002C6
:104AD700BCE0FF25E02400F582E43400F583E0FC28
:104AE700A3E0FDEF25E02402F582E43400F583E03E
:104AF700FEA3E0C39DFFEE9CFECBEFCBFAE4F9F8F3
:104B0700D0E0FFD0E0FED0E0FDD0E0FC122304CDE2
:104B1700EFCDCCEECC9002BCE075F00AA42DFFE5FA
:0F4B2700F03CFE80099002BCE004F0024A20221C
:103F82009002BCEEF0A3EFF09000AAE0F9FDD3EFAF
:103F92009DEE9400500302405B90036EE0FF90029E
:103FA200BCE0FCA3E0FDD39FEC94004078ED946468
:103FB200EC940050709002BCE0FAA3E0FBC374647E
:103FC2009BFFE49AFE7C007D0A1221E1E9FDC3EB2E
:103FD2009DFDEA9CFCD3ED9FEC9E50030240F090C5
:103FE20002BCE0FEA3E0FF9000AAF07C007D0A1272
:103FF20021E19003ABEEF0A3EFF09002BCE0FEA350
:10400200E0FFE4FD90001AE0F8A3E0F9A3E0FAA3D0
:10401200E0FB122279E47B64FAF9F812230490009F
:10402200AB122484229002BCE07004A3E0646460BA
:10403200030240F09000AA7464F09003AB7403F0A2
:10404200A374E8F090001AE0FCA3E0FDA3E0FEA355
:10405200E0FF9000AB122484229000AAE0FD9002BF
:10406200BCE0FEA3E0FFC3ED9FFDE49EFC90034F86
:10407200E0FBD3ED9BEC9400403F9000AAEFF07C74
:10408200007D0A1221E19003ABEEF0A3EFF0900263
:10409200BCE0FEA3E0FFE4FD90001AE0F8A3E0F923
:1040A200A3E0FAA3E0FB122279E47B64FAF9F812A6
:1040B20023049000AB122484229002BCE07002A37D
:1040C200E0702B9000AA04F09003ABE4F0A3740A12
:1040D200F0E47B64FAF9F890001AE0FCA3E0FDA397
:0F40E200E0FEA3E0FF1223049000AB122484221F
:10425A0012370E124A179002BAEEF0A3EFF0E47F7B
:10426A00E87E03FDFC9000ABE0F8A3E0F9A3E0FAD6
:10427A00A3E0FB12227990001AE0F8A3E0F9A3E088
:10428A00FAA3E0FB1223049003ABEEF0A3EFF09045
:10429A0002BAE0FEA3E0FF123F829000AAE0FF7E8E
:1042AA0000900328EEF0FAA3EFF0FB90001AE0FC6E
:1042BA00A3E0FDA3E0FEA3E0FF900346122484CF0F
:1042CA00EBCF7E00E4FCFD900346E0F8A3E0F9A3FF
:1042DA00E0FAA3E0FB122279E47B64FAF9F81223EC
:1042EA00049003791224849000ABE0FCA3E0FDA3C0
:1042FA00E0FEA3E0FF90035B1224849003371224AC
:10430A00A9000000009003A9E0FFA3E090032ECFCC
:10431A00F0A3EFF0E47830F608F67838F608F67885
:10432A0034122490000000009003AF1224A9000068
:10433A000000E490039FF0A3F09003B5F0A3F0907F
:10434A0003ADF0A3F0C25BC257C2599003A8F09024
:10435A0003A7F0783AF608F67832F608F69003AB37
:10436A00E0FFA3E09003B3CFF0A3EFF0C25AC25626
:10437A009003B71224A900000000E49003A9F0A357
:10438A00F09003911224A90000000090039A1224CD
:10439A00A9000000009003951224A900000000E47F
:1043AA0090039EF0900399F0C25890038D1224A9AD
:0843BA0000000000126BE82274
:104D1400124A179002BAEEF0A3EFF0900334E0FFCA
:104D2400E4FCFDFE90001AE0F8A3E0F9A3E0FAA386
:104D3400E0FB122279E47B0AFAF9F8122304C8ECA6
:104D4400C8C9EDC9CAEECACBEFCB90037EE0FCA381
:104D5400E0FDA3E0FEA3E0FFD31223C75003024DFE
:104D6400EA90037DE0FF7E009002BAE0FCA3E0FD40
:104D7400D39FEC9E4070D3900383E0951D900382F3
:104D8400E0951C4061ED9FFBEC9EFA9003ABE0FEC6
:104D9400A3E0FF7C007D0A1221F3C3EF9BEE9A503F
:104DA40045900371E0FFC39002BBE09FFF9002BAFD
:104DB400E09400FE7C007D0A1221E19003ABEEF04A
:104DC400A3EFF0E4FD90001AE0F8A3E0F9A3E0FA01
:104DD400A3E0FB122279E47BE87A03F9F8122304B6
:074DE4009000AB12248422B1
:1025590012370E900343E0FEA3E0FFD3900378E027
:102569009F900377E09E401EE4FFFEFDFC90039AD6
:10257900E0F8A3E0F9A3E0FAA3E0FBD31223B1400A
:1025890005301802D25BC3900383E0951D90038246
:10259900E0951C5012900399E004F0E09405400E78
:1025A9007405F0D2578007C257E4900399F0900060
:1025B90028E0FEA3E0FFEE3395E0FDFC90037EE00A
:1025C900F8A3E0F9A3E0FAA3E0FBD31223B1500387
:1025D9000227C1E49003B5F0A3F09003ADF0A3F096
:1025E90090039EE004F0E0D3940540057405F0D211
:1025F900589000B9E06010D25AE4F09003B7122461
:10260900A900000000C256900375E0FEA3E0FFEEAA
:102619003395E0FDFC900281E0F8A3E0F9A3E0FA2C
:10262900A3E02FFFEA3EFEE93DFDE83CFC90039163
:10263900122484E4FFFEFDFC900391E0F8A3E0F985
:10264900A3E0FAA3E0FBD31223B14021900281E079
:10265900A3E0A3E0FEA3E0FF900376E02FFF900341
:1026690075E03EFE783BEF26F618EE36F6C3783B6A
:10267900E6941018E6940E500302270B0874F0260E
:10268900F61874F136F690001AE0FCA3E0FDA3E019
:10269900FEA3E0FF9000ABE0F8A3E0F9A3E0FAA302
:1026A900E0FBC31223C750219000ABE0FCA3E0FD7F
:1026B900A3E0FEA3E02401FFE43EFEE43DFDE43C8B
:1026C900FC9000AB122484801490001AE0FCA3E073
:1026D900FDA3E0FEA3E0FF9000AB122484305A8DE5
:1026E9009003B7E0FCA3E0FDA3E0FEA3E02401FF13
:1026F900E43EFEE43DFDE43CFC9003B71224840271
:102709002676900343E0FEA3E0FFD3900378E09F91
:10271900900377E09E404490006AE0FEA3E0FFEE5C
:102729003395E0FDFC900281E0F8A3E0F9A3E0FA1B
:10273900A3E0FBC31223B15022C3900069E0951DA9
:10274900900068E0951C501390006CE0FF9003A87E
:10275900E004F0C39F4004EFF0D25B90006AE0FE12
:10276900A3E0FFEE3395E0FDFC900281E0F8A3E0E1
:10277900F9A3E0FAA3E0FBC31223B150359003504B
:10278900E0FCA3E0FDA3E0FEA3E0FF900330E0F846
:10279900A3E0F9A3E0FAA3E0FBC31223C750139007
:1027A9000366E0FF9003A7E004F0C39F4004EFF045
:1027B900D259124D14022AFF900028E0FEA3E0FF2F
:1027C900C3E49FFFE49EFE3395E0FDFC90037EE0A9
:1027D900F8A3E0F9A3E0FAA3E0FBC31223B1400395
:1027E9000229B6E49003A8F09003A7F0C259C25B8E
:1027F9009003ADF0A3F09003B6F090039EF0C25899
:10280900900362E0FCA3E0FDA3E0FEA3E0FF9002D9
:1028190081E0F8A3E0F9A3E0FAA3E02FFBEA3EFA8E
:10282900E93DF9E83CF8900375E0FEA3E0FFEE33DB
:1028390095E0FDFCEB2FFFEA3EFEE93DFDE83CFC9F
:10284900900391122484900391E0FCA3E0FDA3E09E
:10285900FEA3E0FFEC33500AC37833E69FF618E68F
:102869009EF6C37833E6941018E6940E50030229B5
:102879004BC37833E6941018E6940E40670874F059
:1028890026F61874F136F69000B3E0FCA3E0FDA338
:10289900E0FEA3E02401FFE43EFEE43DFDE43CFC50
:1028A9009000B3122484E47F01FEFDFC9000ABE0AC
:1028B900F8A3E0F9A3E0FAA3E0FBD31223C740B1E0
:1028C9009000ABE0FCA3E0FDA3E0FEA3E024FFFF42
:1028D900EE34FFFEED34FFFDEC34FFFC9000AB124B
:1028E9002484808D90001EE0FCA3E0FDA3E0FEA3FC
:1028F900E0FF9000B3E0F8A3E0F9A3E0FAA3E0FB5E
:10290900C31223C7403C9000B3E0FCA3E0FDA3E061
:10291900FEA3E0FF90001EE0F8A3E0F9A3E0FAA30C
:10292900E0FBEF9BFFEE9AFEED99FDEC98FC900021
:10293900B3122484900023E004F07006900022E092
:1029490004F0900354E0FEA3E0FFD3900378E09FE6
:10295900900377E09E5003022AFF9000AFE0FCA3AA
:10296900E0FDA3E0FEA3E0FF900281E0F8A3E0F917
:10297900A3E0FAA3E0FBD31223B15003022AFFD349
:1029890090007BE0951B90007AE0951A5003022A8B
:10299900FF90007CE0FF9003B5E004F09F50030234
:1029A9002AFFEFF09000B97401F0022AFF90037535
:1029B900E0FAA3E0FBFFCEEACEEE3395E0FDFC336F
:1029C9004003022AA9C37833E69BFF18E69AFEF66C
:1029D90008EFF6C39410EE940E5003022AA974F07E
:1029E90026F61874F136F69000B3E0FCA3E0FDA3D7
:1029F900E0FEA3E02401FFE43EFEE43DFDE43CFCEF
:102A09009000B3122484E47F01FEFDFC9000ABE04A
:102A1900F8A3E0F9A3E0FAA3E0FBD31223C740220D
:102A29009000ABE0FCA3E0FDA3E0FEA3E024FFFFE0
:102A3900EE34FFFEED34FFFDEC34FFFC9000AB12E9
:102A4900248490001EE0FCA3E0FDA3E0FEA3E0FFC8
:102A59009000B3E0F8A3E0F9A3E0FAA3E0FBC31206
:102A690023C7403C9000B3E0FCA3E0FDA3E0FEA334
:102A7900E0FF90001EE0F8A3E0F9A3E0FAA3E0FB71
:102A8900EF9BFFEE9AFEED99FDEC98FC9000B312D6
:102A99002484900023E004F07006900022E004F002
:102AA90090038CE0FF9003ADE475F001122248FC1D
:102AB900C3E5F09FEC9400403A900354E0FEA3E094
:102AC900FFD3900378E09F900377E09E4025D39051
:102AD900007BE0951B90007AE0951A401690007CE7
:102AE900E0FF9003B6E004F09F4008EFF09000B9D2
:102AF9007401F01230A6E47FE87E03FDFC9000AB80
:102B0900E0F8A3E0F9A3E0FAA3E0FB122279900030
:102B19001AE0F8A3E0F9A3E0FAA3E0FB122304907A
:102B290003ABEEF0A3EFF0900028E0FEA3E0FFC3B3
:102B3900E49FFFE49EFE3395E0FDFC90037EE0F800
:102B4900A3E0F9A3E0FAA3E0FBC31223B1400C20F0
:102B59001509201A06201B03301C02C25A121056EE
:102B69009000AAE0FF7E00900328EEF0FAA3EFF0B0
:102B7900FB90001AE0FCA3E0FDA3E0FEA3E0FF90B8
:102B89000346122484CFEBCF7E00E4FCFD9003467C
:102B9900E0F8A3E0F9A3E0FAA3E0FB122279E47BD1
:102BA90064FAF9F81223049003791224849000221C
:102BB900E0FFA3E0900367CFF0A3EFF09003ABE051
:102BC900FFA3E09003B3CFF0A3EFF0900391E0FCF3
:102BD900A3E0FDA3E0FEA3E0FF90039A12248490F2
:102BE90000ABE0FCA3E0FDA3E0FEA3E0FF90035BE4
:102BF9001224849003AFE0FCA3E0FDA3E0FEA3E070
:102C0900FF9003371224849003A9E0FFA3E0900307
:0A2C19002ECFF0A3EFF0126BE822BB
:1077490012370E90038D12244390032AE0F8A3E028
:10775900F9A3E0FAA3E0FBC31223C7501490032A4C
:10776900E0FCA3E0FDA3E0FEA3E0FF90038D12245B
:0577790084126BE82200
:1032FE009005F7E4F0A37464F012370E124A17909B
:10330E0005F7EEF0A3EFF04E702E9000AA04F090A9
:10331E0003ABE4F0A3740AF0E47B64FAF9F89000CE
:10332E001AE0FCA3E0FDA3E0FEA3E0FF122304904D
:10333E0000AB12248402340890032AE0FCA3E0FDC3
:10334E00A3E0FEA3E0FF90038DE0F8A3E0F9A3E075
:10335E00FAA3E0FBC31223C7400E9005F7E0FEA3CD
:10336E00E0FF123F82023408E47F64FEFDFC900011
:10337E001AE0F8A3E0F9A3E0FAA3E0FB1222799099
:10338E0000ABE0F8A3E0F9A3E0FAA3E0FB122304FC
:10339E00C8ECC8C9EDC9CAEECACBEFCB90034FE05B
:1033AE00FF9005F8E02FFF9005F7E03400FEE4FCF7
:1033BE00FDD31223C740439005F7E0FAA3E0FB7C50
:1033CE00007D0AFFCEEACE1221E19003ABEEF0A310
:1033DE00EFF0CFEBCFCEEACEE4FD90001AE0F8A3EB
:1033EE00E0F9A3E0FAA3E0FB122279E47B64FAF998
:1033FE00F81223049000AB122484E47830F608F619
:10340E007838F608F6783412249000000000900305
:10341E00AF1224A900000000E490039FF0A3F090E7
:10342E0003B5F0A3F09003ADF0A3F0C25BC257C298
:10343E00599003A8F09003A7F0783AF608F6783280
:10344E00F608F69003ABE0FFA3E09003B3CFF0A332
:10345E00EFF0C25AC2569003B71224A90000000022
:10346E00E49003A9F0A3F09003911224A9000000A8
:10347E000090039A1224A9000000009003951224D4
:10348E00A900000000E490039EF0900399F0C2584A
:10349E0090038D1224A9000000009000AAE0FF7E88
:1034AE0000900328EEF0FAA3EFF0FB90001AE0FC78
:1034BE00A3E0FDA3E0FEA3E0FF900346122484CF19
:1034CE00EBCF7E00E4FCFD900346E0F8A3E0F9A309
:1034DE00E0FAA3E0FB122279E47B64FAF9F81223F6
:1034EE00049003791224849000ABE0FCA3E0FDA3CA
:1034FE00E0FEA3E0FF90035B1224849003371224B6
:10350E00A900000000E490032EF0A3F0126BE82255
:1030A600305A09305B06C25AD2568021305B1E90D8
:1030B60003AB7403F0A374E8F090001AE0FCA3E0FD
:1030C600FDA3E0FEA3E0FF9000AB1224843056037C
:1030D6000231569000B7E0FCA3E0FD900022E0FE2E
:1030E600A3E0FFC39DFDEE9CFCC3900360E09D90B2
:1030F600035FE09C40030232FD205B030232FD12B7
:103106006813E4FCFDFE90001AE0F8A3E0F9A3E0E2
:10311600FAA3E0FB122279ECC0E0EDC0E0EEC0E0DD
:10312600EFC0E09000B7E0FEA3E0FF126813CBEF1C
:10313600CBE4FAF9F8D0E0FFD0E0FED0E0FDD0E035
:10314600FC1223049003B71224840232B20232B274
:10315600C256E47F32FEFDFC900016E0F8A3E0F9CB
:10316600A3E0FAA3E0FB122279E47B64FAF9F812F1
:1031760023049002BA1224849002BAE0FCA3E0FD74
:10318600A3E0FEA3E0FF9003B7E0F8A3E0F9A3E015
:10319600FAA3E02FFFEA3EFEE93DFDE83CFC900085
:1031A60016E0F8A3E0F9A3E0FAA3E0FBC31223C7F5
:1031B60040030232FD900345E0FFE4FCFDFE900073
:1031C6001AE0F8A3E0F9A3E0FAA3E0FB122279E4FF
:1031D6007B64FAF9F81223049002BA12248490024E
:1031E600BAE0FCA3E0FDA3E0FEA3E0FF90001AE036
:1031F600F8A3E0F9A3E0FAA3E02FFFEA3EFEE93DDB
:10320600FDE83CFC9003B7E0F8A3E0F9A3E0FAA3DD
:10321600E0FBD31223C7402E9002BAE0FCA3E0FDE8
:10322600A3E0FEA3E0FF90001AE0F8A3E0F9A3E014
:10323600FAA3E02FFFEA3EFEE93DFDE83CFC9003E1
:10324600B712248480669002BAE0FCA3E0FDA3E0F6
:10325600FEA3E0FF9003B7E0F8A3E0F9A3E0FAA32A
:10326600E02FFFEA3EFEE93DFDE83CFC90001AE057
:10327600F8A3E0F9A3E0FAA3E0FBD31223C7402C9E
:103286009002BAE0F8A3E0F9A3E0FAA3E0FB90000D
:103296001AE0FCA3E0FDA3E0FEA3E09BFFEE9AFE8E
:1032A600ED99FDEC98FC9003B71224849003B7E0E7
:1032B600FCA3E0FDA3E0FEA3E0FF90001A12248425
:1032C6009003AB7403F0A374E8F090001AE0FCA33B
:1032D600E0FDA3E0FEA3E0FF9000AB122484900083
:1032E60022E0FFA3E09000B7CFF0A3EFF09003B782
:0832F6001224A90000000022CF
:10681300C3900389E09F900388E09E5004795580DC
:1068230048C3900387E09F900386E09E5016900331
:106833004CE0FCA3E0FD1221F390033DE0A3E0C391
:106843009FF98025C3900385E09F900384E09E50C9
:106853001690034AE0FCA3E0FD1221F390033BE012
:0D686300A3E0C39FF980027964CFE9CF2242
:10105600E49002BAF0A3F0FFA3F0A3F0A3F090038C
:10106600A1E0645A6028A2AF924DC2AF75A701E411
:10107600EF90124093FE74A12FF582E43403F583BA
:10108600EEF00FEFB406E9E4F5A7A24D92AF900398
:10109600A6E064C36003021C48FF74A12FF582E436
:1010A6003403F583E0FEEF907D0F936E6003021C20
:1010B600480FEFB406E48003021C48900028E0FEC7
:1010C600A3E0FFEE3395E0FDFC90037EE0F8A3E09D
:1010D600F9A3E0FAA3E0FBD31223B150030214F103
:1010E6002058030214F1E47830F608F67838F6084A
:1010F600F69000AAE0D394634003021C48C3900311
:1011060083E0951D900382E0951C401E90034EE0FF
:10111600FF7E007C007D0A1221E1D39003ACE09FA4
:101126009003ABE09E50030213C930575A90034E0A
:10113600E0FBFF7E007C007D0A1221E19003ACE01B
:101146002496FD9003ABE03400FCC3ED9FEC9E506B
:1011560036EBFF7E007C007D0A1221E1EEF0A3EF64
:10116600F0CFEBCFE4FDFE90001AE0F8A3E0F9A380
:10117600E0FAA3E0FB122279E47B64FAF9F8122381
:10118600049000AB122484900350E0FCA3E0FDA37E
:10119600E0FEA3E0FF900330E0F8A3E0F9A3E0FA55
:1011A600A3E0FBD31223C75003021230900350E092
:1011B600F8A3E0F9A3E0FAA3E0FB900330E0FCA378
:1011C600E0FDA3E0FEA3E09BFBEE9AFAED99F9ECB5
:1011D60098F890038AE0FFE4FCFDFE122279E47B96
:1011E6000AFAF9F8122279EEC0E0EFC0E090001496
:1011F600E0FEA3E0FFC3900069E09FFF900068E077
:101206009EFECBEFCBFAE4F9F8D0E0FFD0E0FE1279
:101216002304EFC0E0AF13CBEFCBE4FAF9F8D0E04C
:10122600FF122304900395122484C3900063E09573
:101236001DFF900062E0951CFE90038AE0FD7C0095
:1012460012252CE47B0AFAF9F8122279EEC0E0EFB7
:10125600C0E0900014E0FEA3E0FFC3900069E09FA9
:10126600FF900068E09EFECBEFCBFAE4F9F8D0E001
:10127600FFD0E0FE1223049002BF1224849003954F
:10128600E0FCA3E0FDA3E0FEA3E0FF9002BFE0F8D0
:10129600A3E0F9A3E0FAA3E0FBC31223C75014901E
:1012A60002BFE0FCA3E0FDA3E0FEA3E0FF900395F0
:1012B600122484E47F24FEFDFC90001AE0F8A3E0EB
:1012C600F9A3E0FAA3E0FB122279900395E0F8A3D4
:1012D600E0F9A3E0FAA3E0FB122279EEC0E0EFC04A
:1012E600E09000AAE0FFC374659FFFE49400FECB84
:1012F600EFCBFAE4F9F8D0E0FFD0E0FE122304E4E5
:101306007B0AFAF9F81223049003951224849000BC
:101316006AE0FEA3E0FFEE3395E0FDFC900391E06A
:10132600F8A3E0F9A3E0FAA3E0FBD31223B1406CE3
:10133600900391E0FCA3E0FDA3E0FEA3E0FFC8EC70
:10134600C8A3E0FCA3E0FDA3E0FEA3E0FF12230494
:10135600ECC0E0EDC0E0EEC0E0EFC0E090006AE077
:10136600FEA3E0FFFBCAEECAEA3395E0F9F8900364
:1013760091E0FCA3E0FDA3E0FEA3E0C39BFFEE9A91
:10138600FEED99FDEC98FCD0E0FBD0E0FAD0E0F958
:10139600D0E0F8122279900395122484900063E03D
:1013A60024FFFF900062E034FFFEC3E51D9FE51CAD
:1013B6009E50030214839003951224A90000000096
:1013C6000214839003ABE0FEA3E0FF7C007D0A12CB
:1013D60021F3EF2401FFE43EFE9000AAE0FB7A0031
:1013E600C39FEA9E503C9003ABE0FEA3E0FF7C0067
:1013F6007D0A1221F3EB2401FDEA33FCD3ED9FECC9
:101406009E401FE47F24FEFDFC90001AE0F8A3E056
:10141600F9A3E0FAA3E0FB12227990039512248443
:10142600805B9000ABE0F8A3E0F9A3E0FAA3E0FB51
:1014360090001AE0FCA3E0FDA3E0FEA3E0C39BFF3F
:10144600EE9AFEED99FDEC98FCE47B107A0EF9F825
:10145600122279EEC0E0EFC0E09000AAE0FFC3746C
:10146600649FFFE49400FECBEFCBFAE4F9F8D0E0FA
:10147600FFD0E0FE1223049003951224849003917A
:10148600E0FCA3E0FDA3E0FEA3E0FFFBCAEECAC9B1
:10149600EDC9C8ECC8A3E0FCA3E0FDA3E0FEA3E011
:1014A600FF1223049002BDEEF0A3EFF020590330A3
:1014B6005B0D90038BE0FF9002BDE4F0A3EFF0908C
:1014C60003A9E475F001122248FEC39002BEE0951E
:1014D600F09002BDE09E4003021C489000AAE00482
:1014E600F0E49003A9F0A3F0021C48900028E0FE67
:1014F600A3E0FFC3E49FFFE49EFE3395E0FDFC906E
:10150600037EE0F8A3E0F9A3E0FAA3E0FBC312230D
:10151600B14003021BE89000AAE094015003021CAC
:1015260048900326E0FEA3E0FFAD137C0012252CB5
:10153600900350E0F8A3E0F9A3E0FAA3E0FBC3129E
:1015460023C7402DD390007BE0951B90007AE09551
:101556001A501E90035AE0FF7E007C007D0A12217D
:10156600E1C39003ACE09F9003ABE09E40030218FA
:101576000B90036FE0FEA3E0FFD3900378E09F900B
:101586000377E09E500302180B900369E0FCA3E08A
:10159600FDA3E0FEA3E0FF90037EE0F8A3E0F9A33D
:1015A600E0FAA3E0FBD31223B1500302180B7839FB
:1015B600E61846700302180B90039AE0FCA3E0FDC0
:1015C600A3E0FEA3E024D0FFEE3407FEE43DFDE4F5
:1015D6003CFC900391E0F8A3E0F9A3E0FAA3E0FB5A
:1015E600C31223B1400302180B90039AE0FCA3E058
:1015F600FDA3E0FEA3E02430FFEE34F8FEED34FF59
:10160600FDEC34FFFC900391E0F8A3E0A3E0A3E037
:10161600D31223B1500302180B900361E07E00251C
:101626001BFFEE351AFEC3EF783996EE1896400387
:101636000217FA90039FE0FEA3E0FF9400EE9400E9
:1016460050030217FAEF9401EE9400500890039F9E
:10165600E4F0A304F0900350E0FCA3E0FDA3E0FE59
:10166600A3E0FF783412242AD31223C750030217AB
:1016760013900356E0F8A3E0F9A3E0FAA3E0FB9089
:101686000350E0FCA3E0FDA3E0FEA3E09BFBEE9A83
:10169600FAED99F9EC98F890039FE0FEA3E0FFE4D9
:1016A600FCFD122279ECC0E0EDC0E0EEC0E0EFC038
:1016B600E0900350E0F8A3E0F9A3E0FAA3E0FBE82A
:1016C600C0E07834122412D0E0F8C3EF9BFBEE9A08
:1016D600FAED99F9EC98F8D0E0FFD0E0FED0E0FD05
:1016E600D0E0FC122304EEC0E0EFC0E09000AAE0D8
:1016F60024FFFFE434FFFECBEFCBFAE4F9F8D0E0A9
:10170600FFD0E0FE12230490039512248490007407
:10171600E0FEA3E0FFC3E51B9FFFE51A9EFE9003D4
:101726009FE0FCA3E0FD12252CEEC0E0EFC0E0C375
:101736007839E6951BFF18E6951AFECBEFCBFAE44F
:10174600F9F8D0E0FFD0E0FE122304EEC0E0EFC0CF
:10175600E09000AAE024FFFFE434FFFECBEFCBFAD3
:10176600E4F9F8D0E0FFD0E0FE1223049002BF12A5
:101776002484900395E0FCA3E0FDA3E0FEA3E0FF34
:101786009002BFE0F8A3E0F9A3E0FAA3E0FBC312DE
:1017960023C750149002BFE0FCA3E0FDA3E0FEA324
:1017A600E0FF9003951224847838A61A08A61B90A9
:1017B6000350E0FCA3E0FDA3E0FEA3E0FF783412B3
:1017C6002478E490039FF0A3F0900395E0F8A3E05B
:1017D600F9A3E0FAA3E0FB900391E0FCA3E0FDA3EC
:1017E600E0FEA3E0FF1223A31222799003951224B0
:1017F60084021B769003A0E004F0700690039FE03D
:1018060004F0021B767838A61A08A61B900350E04F
:10181600FCA3E0FDA3E0FEA3E0FF7834122478E405
:1018260090039FF0A3F090036FE0FEA3E0FFC39048
:101836000378E09F900377E09E4021900369E0FCE7
:10184600A3E0FDA3E0FEA3E0FF90037EE0F8A3E0A3
:10185600F9A3E0FAA3E0FB1223B1501D90001AE0B1
:10186600FCA3E0FDA3E0FEA3E0FF9003AF122484F7
:10187600E47830F608F60219FA7830E6FE08E6FF54
:101886002414FDE43EFC900377E0FAA3E0FBD39D2D
:10189600EA9C5011EB2414FDE43AFCD3EF9DEE9C38
:1018A60050030219FA900377E0FEA3E0FF7830EECA
:1018B600F608EFF62487FFEE34F59002BAF0A3EFB0
:1018C600F0900341E0FEA3E0FFFBCAEECAE4F9F89C
:1018D6009002BAE0FEA3E0FFEE3395E0FDFC122293
:1018E60079C8ECC8C9EDC9CAEECACBEFCB90033FA5
:1018F600E0FEA3E0FFE4C3EF9BFBEE9AFAE499F95E
:10190600E498F89002BAE0FEA3E0FFEE3395E0FD1E
:10191600FC122279E47B107A27F9F8127380C8EC5E
:10192600C8C9EDC9CAEECACBEFCB900373E0FEA3DC
:10193600E0FFE4FCFDEB2FFFEA3EFEED39FDEC385F
:10194600FC90001AE0F8A3E0F9A3E0FAA3E0FB128A
:101956002279E47BD07A07F9F81223049003AF12B8
:10196600248490001AE0FCA3E0FDA3E0FEA3E0FFC0
:101976009003AFE0F8A3E0F9A3E0FAA3E0FBD312EB
:1019860023C7401690001AE0FCA3E0FDA3E0FEA3E7
:10199600E0FF9003AF122484805AE47F06FEFDFC2C
:1019A60090001AE0F8A3E0F9A3E0FAA3E0FB122204
:1019B60079E47B0AFAF9F81223049003AFE0F8A35E
:1019C600E0F9A3E0FAA3E0FBC31223C75026E47FA5
:1019D60006FEFDFC90001AE0F8A3E0F9A3E0FAA3E6
:1019E600E0FB122279E47B0AFAF9F8122304900349
:1019F600AF1224849003AFE0F8A3E0F9A3E0FAA3C2
:101A0600E0FB90001AE0FCA3E0FDA3E0FEA3E0C328
:101A16009BFFEE9AFEED99FDEC98FCE47B0DFAF93E
:101A2600F8122279E47B0AFAF9F81223049000AB43
:101A3600E0F8A3E0F9A3E0FAA3E0FBC31223C75042
:101A460020E47F24FEFDFC90001AE0F8A3E0F9A351
:101A5600E0FAA3E0FB122279900395122484021B7C
:101A6600769000ABE0FCA3E0FDA3E0FEA3E0FF90D0
:101A760003AFE0F8A3E0F9A3E0FAA3E02FFFEA3E04
:101A8600FEE93DFDE83CFC90001AE0F8A3E0F9A36E
:101A9600E0FAA3E0FBC3EF9BFFEE9AFEED99FDECA7
:101AA60098FCE47B64FAF9F81222799003AFE0F827
:101AB600A3E0F9A3E0FAA3E0FB1223049002BCEF33
:101AC600F02401FFE433FE9000AAE0FDC39FEE641C
:101AD60080F87480985035ED2401FFE433FE9002BF
:101AE600BCE0FDD3EF9D7480F86E98401FE47F2420
:101AF600FEFDFC9003AFE0F8A3E0F9A3E0FAA3E053
:101B0600FB12227990039512248480649000ABE046
:101B1600FCA3E0FDA3E0FEA3E0FF9003AFE0F8A383
:101B2600E0F9A3E0FAA3E02FFFEA3EFEE93DFDE877
:101B36003CFC90001AE0F8A3E0F9A3E0FAA3E0FB6E
:101B4600C3EF9BFFEE9AFEED99FDEC98FCE47B104B
:101B56007A0EF9F8122279EFC0E09000AAE0FFFBB6
:101B6600E4FAF9F8D0E0FF122304900395122484D6
:101B7600900391E0FCA3E0FDA3E0FEA3E0FF1223A7
:101B8600A3CBEFCBCAEECAC9EDC9C8ECC8A3E0FC2B
:101B9600A3E0FDA3E0FEA3E0FF1223049002BDEE46
:101BA600F0A3EFF09003A9E475F001122248FCD3EC
:101BB600E5F09FEC9E400D9000AAE014F0E490033F
:101BC600A9F0A3F030197B900372E0FF9000AAE021
:101BD600D39F506E90036DE060689000AA7401F088
:101BE6008060E47838F608F6783412249000000015
:101BF60000E47830F608F69000AAE0D3940140425B
:101C0600900375E0FEA3E0FFEE3395E0FDFC335054
:101C1600319003ABE0FEA3E0FF7C007D0A1221F3C6
:101C2600CAEECACBEFCB9003B3E0FEA3E0FF7C0085
:101C36007D0A1221F3D3EF9BEE9A40069000AAE0AC
:101C460014F0E4FFFEFDFC90039AE0F8A3E0F9A38C
:101C5600E0FAA3E0FBD31223B14009301806900046
:101C6600AA7464F09002BDE0FFA3E0900335CFF0C4
:041C7600A3EFF022C6
:107AB100304C19204306204403304510C24CC243C8
:0D7AC100C244C245C2AF127C261200A622AC
:10000000020D7A021003000000000002100B000035
:10001000000000021013000000000002101B00008E
:10002000000000021023000000000002102B00005E
:10003000000000021033000000000002103B00002E
:10004000000000021043000000000002104B0000FE
:10005000000000021053000000000002105B0000CE
:10006000000000021063000000000002106B00009E
:10007000000000021073000000000002107B00006E
:10008000000000021083000000000002108B00003E
:10009000000000021093000000000002109B00000E
:1000A0000000000210A3E4F526F525F524F523F55C
:1000B00030F52FF52EF52DF52C120D5E209803024C
:1000C000018E7400252BF582E43402F583E599F066
:1000D000052BE52BC3948C4003E4F52BE52BB401F1
:1000E0000D900200E0645A700302018C806BE52BD6
:1000F000B40214900201E064A56002805CE4F53172
:10010000F532F52202018C900202E0FF7E00240904
:10011000FDEE33FCAB2B7A00C3EB9DEC6480F874EE
:1001200080985062EF2407FFEE33FED3EB9FEE641E
:1001300080F8748098501574FF252BF582E4340103
:10014000F583E02532F532E43531F531E52BB405A0
:100150000D900204E064076033E4F52B802EE52B5C
:1001600064067028900205E0FF6406601FEF6407D4
:10017000601AEF64086015EF64096010EF640A60AC
:100180000B432230800653B1F8120A9DC298309971
:100190004453B1F8900202E02408FFE433FEC3E5C3
:1001A0002B9FEE6480F87480984013E4F586D29C0F
:1001B000F52B900200F0A3F0A3F0D2028015052BDE
:1001C000E4F586C29C7400252BF582E43402F583A5
:1001D000E0F599C299E52C640A60030200BC53B1B2
:1001E000F82002030200BCC202F52C12000002003B
:1001F000BCC200900206E0FFC395214014E5212413
:1002000004FDE433FCD3EF9DEC6480F874809840E7
:100210000A900206E060047405F022900206E0F500
:1002200021E4F0900202E070152526F526E525343C
:1002300002F525E43524F524E43523F52322E521D0
:100240005403F50AE4F508F509900202E0FD7C008C
:10025000C3E5099DE5089C503274072509F582E441
:100260003402F583E0FBAF0A7E00120638E5092F61
:10027000FFE5083EFE74002FF58274003EF583EB27
:10028000F00509E50970C2050880BEE50A6403604F
:100290000302044F751D551208955003020386E4AE
:1002A000FF7E02FDFCAB26AA25A924A8231207186D
:1002B000401AE5269400F526E5259402F525E52467
:1002C0009400F524E5239400F5238009E4F526F550
:1002D00025F524F523E4F50F30015E2526F50EE51E
:1002E000253410F50DE43524F50CE43523F50BE445
:1002F000252AFFE529340CFEE43528FDE43527FCEA
:10030000AB0EAA0DA90CA80BC31207184040E42598
:100310002AFBE529340CFAE43528F9E43527F8C33B
:10032000E50E9BF50EE50D9AF50DE50C99F50CE53E
:100330000B98F50B750F018015E42526F50EE525C4
:100340003484F50DE43524F50CE43523F50B751DE7
:1003500055AF0EAE0DAD0CAC0B850F15120B7EAF6D
:100360000EAE0DAD0CAC0B850F15120C8C500E1291
:10037000089540129002067403F002044C900206A5
:100380007402F002044CE4F50A75F004E50AA424B2
:1003900002F582E5F03400F583E0FFE4FCFDFE7831
:1003A0001012073CC004C005C006C00775F004E584
:1003B0000AA42403F582E5F03400F583E0FFE4FCB1
:1003C000FDFE781812073CD003D002D001D000EF18
:1003D0004BFFEE4AFEED49FDEC48FCC004C005C0F1
:1003E00006C00775F004E50AA42401F582E5F0349F
:1003F00000F583E0FFE4FCFDFE780812073CD00323
:10040000D002D001D000EF4BFBEE4AFAED49F9ECF7
:1004100048F875F004E50AA42400F582E5F03400FC
:10042000F583E0FFEB4FFFEAFEE9FDE8FCE5302F46
:10043000F530E52F3EF52FE52E3DF52EE52D3CF56B
:100440002D050AE50A64806003020389E4F51D2294
:10045000E4F526F525F524F523F530F52FF52EF5F1
:100460002DF52AF529F528F527900209E0FFE4FC8F
:10047000FDFE781012073CC004C005C006C007A3EB
:10048000E0FFE4FCFDFE781812073CD003D002D058
:1004900001D000EF4BFFEE4AFEED49FDEC48FCC0F9
:1004A00004C005C006C007900208E0FFE4FCFDFEA2
:1004B000780812073CD003D002D001D000EF4BFBEC
:1004C000EE4AFAED49F9EC48F8900207E0FFEB4FED
:1004D000F52AEAF529E9F528E8F527200006900233
:1004E00006740AF0E4FF7E78FDFCAB2AAA29A9284D
:1004F000A827D312071840052001028017E4FF7EC9
:10050000ECFDFCAB2AAA29A928A827D3120718407A
:100510000A3001079002067401F022E4900206F00E
:10052000F521751D55F515FF7E0EFDFC120B7EE4C1
:10053000F515FF7E0EFDFC120C8C502B30012E7534
:100540001BA5E4F51C7FFF7E0FFDFC120B15E4F5E7
:100550001B7FFF7E0FFDFC120D94EF64A5600E90D3
:1005600002067403F080069002067402F0E4F51DA2
:10057000900206E06003020631FB7A02F9F8AF2A26
:10058000AE29AD28AC271206868F09E4F508E508E8
:10059000C395094003020637E4F50A300107F50E5A
:1005A000750D108006E4F50E750D84F50CF50BE560
:1005B0000825E0FEE4FCFD250EF50EE50D3EF50DEB
:1005C000ED350CF50CEC350BF50B300135E5092458
:1005D000FEFBE434FFFAED34FFF9EC34FFF8AF082A
:1005E000E4FED3120718501A750A01E5082402FF29
:1005F000C3EF9509FFEF25E0FEE4F50E8E0DF50C37
:10060000F50B751D55AF0EAE0DAD0CAC0B850A1577
:10061000120B7EAF0EAE0DAD0CAC0B850A15120C95
:100620008C40069002067402F0E4F51D05080205F0
:100630008E9002067405F022EF8DF0A4A8F0CF8C06
:10064000F0A428CE8DF0A42EFE2275F0087582004D
:10065000EF2FFFEE33FECD33CDCC33CCC58233C587
:10066000829BED9AEC99E58298400CF582EE9BFE18
:10067000ED9AFDEC99FC0FD5F0D6E4CEFBE4CDFA73
:10068000E4CCF9A88222B800C1B90059BA002DEC17
:100690008BF084CFCECDFCE5F0CBF97818EF2FFFAF
:1006A000EE33FEED33FDEC33FCEB33FB10D7039957
:1006B0004004EB99FB0FD8E5E4F9FA227818EF2F04
:1006C000FFEE33FEED33FDEC33FCC933C910D70523
:1006D0009BE99A4007EC9BFCE99AF90FD8E0E4C942
:1006E000FAE4CCFB2275F010EF2FFFEE33FEED3372
:1006F000FDCC33CCC833C810D7079BEC9AE899409F
:100700000AED9BFDEC9AFCE899F80FD5F0DAE4CD00
:10071000FBE4CCFAE4C8F922EB9FF5F0EA9E42F044
:10072000E99D42F0E89C45F022E8600FECC313FC21
:10073000ED13FDEE13FEEF13FFD8F122E8600FEF8B
:10074000C333FFEE33FEED33FDEC33FCD8F122EC86
:100750008EF0A4CCC5F0CCCDF8EFA4CEC5F02DFD25
:10076000E43CFCE8A42EC8C5F03DFDE43CFCEFA44D
:10077000FFE5F028FEE43DFDE43CFC22E4F50853EF
:10078000B1F8E508C3943A501FE4F50AAF08FE7CBF
:1007900002FD12074FE42FF510EE3410F50FE43D83
:1007A000F50EE43CF50D8021750A01AF087E007C52
:1007B000027D0012074FE42FF510EE348CF50FED9B
:1007C00034FFF50EEC34FFF50D751D55AF10AE0F6F
:1007D000AD0EAC0D850A15120B7EAF10AE0FAD0E2F
:1007E000AC0D850A15120C8C4003020883E4F50B4E
:1007F000F50CAE0BAF0CE4FCFDFB7A02F9F8D3125A
:1008000007185003020886AF087E007C027D0012A4
:10081000074FA804A905AA06AB07E4250CFFE50BC2
:100820003484FEE433FDE433FCEB2FFFEA3EFEE9C3
:100830003DFDE83CFCE4F51B120D948F09E50C2509
:1008400010FFE50B350FFEE4350EFDE4350DFC859C
:10085000091B850A1C120B15E50C2510FFE50B354D
:100860000FFEE4350EFDE4350DFC850A1B120D94D8
:10087000EF650960037F0222050CE50C7002050B91
:100880000207F27F01220508E508C3943C500302E9
:10089000077F7F0022D203E4F510F511AE10AF11EF
:1008A000E4FCFDFB7A02F9F8D312071850030209A1
:1008B0008CE4F51630015E2526F515E5253410F596
:1008C00014E43524F513E43523F512E4252AFFE575
:1008D00029340CFEE43528FDE43527FCAB15AA14B9
:1008E000A913A812C31207184040E4252AFBE529E2
:1008F000340CFAE43528F9E43527F8C3E5159BF5FF
:1009000015E5149AF514E51399F513E51298F51207
:100910007516018015E42526F515E5253484F514B2
:10092000E43524F513E43523F512AF15AE14AD13F9
:10093000AC1274002511F58274003510F583E0F5D2
:100940001B85161C120B15AF15AE14AD13AC12851A
:10095000161B120D9474002511F58274003510F5E4
:1009600083E06F6004C2038023E5262401F526E4BA
:100970003525F525E43524F524E43523F523051143
:10098000E511600302089C051002089CA203227E68
:10099000007D007C00900209E0FFE4781012073C23
:1009A000C004C005C006C007A3E0FFE4FCFDFE785C
:1009B0001812073CD003D002D001D000EF4BFFEE5D
:1009C0004AFEED49FDEC48FCC004C005C006C00766
:1009D000900208E0FFE4FCFDFE780812073CD0031B
:1009E000D002D001D000EF4BFBEE4AFAED49F9EC12
:1009F00048F8900207E0FFEB4FFFEAFEE9FDE8FC54
:100A0000AB30AA2FA92EA82DC31207186007900299
:100A1000067408F022E4900206F022E4F508F509D5
:100A2000900202F0900205740BF0900203E0FFA325
:100A3000E0900203F0A3EFF07F02900202E0FE24B8
:100A400007FDE433FCEFC39DEC6480F8748098509C
:100A50001774002FF582E43402F583E02509F509C7
:100A6000E43508F5080F80D274072EF582E43402CD
:100A7000F583E509F0E508FF900202E02408F5821D
:100A8000E43402F583EFF0C202E4F586C29C740000
:100A9000252BF582E43402F583E0F59922E4F52B69
:100AA000900202E0FD2408F582E43402F583E0FEC2
:100AB00074072DF582E43402F583E07C002400FF06
:100AC000EC3EFEEF65327003EE6531600343228039
:100AD000E5226006900206F08038900205E0FEB440
:100AE0000605120CD5802BEEB407051204508022A7
:100AF000900205E0B408051201F18016900205E0AD
:100B0000B4090512098F800A900205E0B40A0312A5
:100B10000BDE020A1B8F1A8E198D188C17851CA7E5
:100B2000AF1AAE19AD18AC1778081207298FF7E580
:100B30001AFF8FFB851BFC75F26E20AF3D75F30528
:100B4000E5A7651C703475F40AE51DB4552C75F5E0
:100B500009AF1AAE19AD18AC177808120729A80406
:100B6000A905AA06AB07AFF7E4FCFDFEC312071800
:100B7000700875F6060000000000E4F5A7228F1447
:100B80008E138D128C118515A7AF14AE13AD12AC58
:100B90001178081207298FF775F2E620AF3C75F33C
:100BA00005E5A76515703375F40AE51DB4552B7579
:100BB000F509AF14AE13AD12AC117808120729A8CD
:100BC00004A905AA06AB07AFF7E4FCFDFEC31207B4
:100BD00018700775F60600000000E4F5A722E490FF
:100BE0000206F0752C0A751D55F515FF7E0EFDFCED
:100BF000120B7EE4F515FF7E0EFDFC120C8C502AC4
:100C0000200130751B5AE4F51C7FFF7E0FFDFC129E
:100C10000B15E4F51B7FFF7E0FFDFC120D94EF64B6
:100C20005A6010900206740380059002067402F068
:100C3000E4F52CE4F51D2253B1F8120DACE4F51BDC
:100C40007FFF7E0FFDFC120D94EF645A7026C201E7
:100C5000751D55120D3850028005120D385005E4EF
:100C6000F51D8024E4F51D758E55438702000000B4
:100C7000000080F0E4F51B7FFF7E0FFDFC120D9459
:100C8000BFA505D2010200A6121000228F148E13F8
:100C90008D128C11D2048515A7E4F516F517AE1642
:100CA000AF17E4FCFDFB7A02F9F8D3120718401FD6
:100CB000E5172514FFE51635138F82F583E493605D
:100CC00004C204800A0517E51770D3051680CFE427
:100CD000F5A7A20422E4900206F0A3E0FFB4490FB6
:100CE000A3E0B4410AA3E0B45005C201D20022EF50
:100CF000B44911900208E0B4530AA3E0B45005D2FD
:100D000001D20022900206740AF0C200227580F817
:100D100075E18F75E9C875908075E27F75EA807519
:100D2000A0E075E33F75EBC075B01975E4E675ECAE
:100D3000194380C043E98022D20312077CEF701967
:100D4000F515FF7E0EFDFC120B7EE4F515FF7E0E01
:100D5000FDFC120C8C92038002C203A2032275C414
:100D600032E4F587759850759D7F759C64759E0477
:100D7000439D80759A0A759BFF2275817F75B20825
:100D8000000000000000000043B20478FFE4F6D841
:100D9000FD020C378F1A8E198D188C17E4851BA74E
:100DA000851A8285198393FFE4F5A722120DB512E7
:100DB0000D0DC20022E4F5A8F5A9F5AA2200000055
:100DC0000000000000000000000000000000000023
:100DD0000000000000000000000000000000000013
:100DE0000000000000000000000000000000000003
:100DF00000000000000000000000000000000000F3
:101C7A00021E1CE86480F8E933E83360110460F05E
:101C8A00ED33EC337009E8FCE9FDEAFEEBFF2204D0
:101C9A0060DED3EB9FEA9EE99DE8C2E78CF0C2F7CB
:101CAA0095F0400CE8CCF8E9CDF9EACEFAEBCFFB97
:101CBA00121DE785D0F05804700320D5B3E80470EC
:101CCA00075002B2D5021E2692D5EC0460F7E4CC86
:101CDA00C0E0C398F8603B94186008400DD0E0FB60
:101CEA00021DFEE4FBFAC9FC8028E830E406E4C9D8
:101CFA00FBE4CAFCE830E305E4C9CACBFCE85407B4
:101D0A006010F8C3E913F9EA13FAEB13FBEC13FCBE
:101D1A00D8F130F52FC3E49CFCEF9BFFEE9AFEED61
:101D2A0099FDD0E0FBEF4E4D4C701222DB03021EF0
:101D3A0023EC2CFCEF33FFEE33FEED33FDED30E701
:101D4A00EB021DFEEF2BFFEE3AFEED39FDD0E0FB74
:101D5A0050130BBB0003021E26ED13FDEE13FEEF1C
:081D6A0013FFEC13FC021DFE47
:101D720075F020800E75F010800575F0087D007EEC
:101D8200007F003392D530D5031223A3EC334010E9
:101D9200EF33FFEE33FEED33FDEC33FCD5F0ED22F5
:0E1DA200E5F0247EA2D513CC92E7CDCEFF2231
:101DB000EDD2E7CD33EC3392D524814006E4FFFE2B
:101DC000FDFC22FCE4CFCECDCC24E0501174FF808A
:101DD000EDC3CC13CCCD13CDCE13CECF13CF047027
:071DE000F030D5DE0223A361
:102C2300E51524BDF582E43402F583E00515229011
:102C330002BA3054039002BDE475F0011224E60297
:102C43002189204DE97F2ED24D8018EF540F249017
:102C5300D43440D4FF30510BEF24BFB41A005003D7
:102C63002461FFE516600215160519E519700205C2
:102C73001830540E9002BAE475F0011224E6EF0204
:102C830021CF027CDF7403D2548003E4C254F515D0
:102C93009002BA1224FDE4F516F518F519E516604D
:102CA300077F20122C6680F57517FFC24EC24DC2F6
:102CB3004FC250C252C253C255122C32FF700D3054
:102CC30054057F00122C77AF19AE1822B4255FC2CA
:102CD300D5C251122C32FF24D0B40A00501A75F019
:102CE3000A781630D50508B6FF0106C6A426F620D5
:102CF300D5047002D25080D924CFB41A00EF500407
:102D0300C2E5D251022F69D24E80C6D24D80C0D2C5
:102D13004F80BCD2D580BAD25280B47F20122C66A9
:102D2300204F077401B5160040F1122C23FF122C1B
:102D330066022CA0D255D2538095122C23FB122C61
:102D430023FA122C23F94A4B700679677A307BFFFA
:102D5300204F2EE516602A7E008E82758300122195
:102D6300A260060EEE651770F0C2D5EBC0E0EAC0B4
:102D7300E0E9C0E0EE122FCAD0E0F9D0E0FAD0E0EB
:102D8300FB122189FF60AAEBC0E0EAC0E0E9C0E0E2
:102D9300122C66D0E02401F9D0E03400FAD0E0FB35
:102DA300E5170460DCD517D98087D24F80A2122F94
:102DB300AC60F7E517700104121E31A917600DE529
:102DC30017600914F517123054EF60F3EA30E70285
:102DD300F404C3995079EAF425170430E701E404B5
:102DE300F517800D122FAC60C1EA05172517121EC7
:102DF30031EA9002E9F030E701E4251704D517041E
:102E030020520114122FCAE4C0E01230549002E998
:102E1300E0601320E70714F0122C4E802204F0D058
:102E2300E014C0E07F00122C4EE5176007122C451A
:102E33001517800B305203122C45D0E0022CA0D082
:102E4300E00480C4122FAC609EE51704121E31907B
:102E530002E9EAF0E5172052026001042404122F6C
:012E6300CAA4
:102E640074FF04C0E0123054122C4EE517205202B5
:102E74006003122C45D0E0B517E87F45122C58901A
:102E840002E9E07F2B30E7047F2DF404C0E0122C2C
:102E940066D0E075F00A84C0F0122C4FD0E0122CFA
:102EA4004F022CA0791080027908C253C2558008C1
:102EB400D2D5790A8004790AC2D5E517047002F5DF
:102EC40017E4FAFDFEFF122C23FC7B08204E13129C
:102ED4002C23FD7B10304D0A122C23FE122C23FFD1
:102EE4007B20EC3382D592D55013C3E4304D069F3A
:102EF400FFE49EFEE4204E039DFDE49CFCE4CBF83D
:102F0400C24EEC700CCFCECDCCE824F8F870F38030
:102F140017C3EF33FFEE33FEED33FDEC33FCEB333D
:102F2400FB994002FB0FD8E9EB304E05F8D0E0C422
:102F340048B24EC0E00AEC4D4E4F78207B0070C280
:102F4400EAB5170040BCC0E0122FCCD0F0D0E0208E
:102F54004E04C4C0E0C4B24EC0F0122C4FD0F0D521
:102F6400F0EB022CA01225062D3D532EA8582D0E51
:102F74004C2D0A422EAC4F2EB4442EB4492D23437B
:102F84002EBA552DE7462E47452DB1473087502D93
:102F9400122D2D162E2D392B2D1A232D372030705E
:102FA4002A2CD24800002D31E517B4FF037517060B
:102FB400122C23FC122C23FD122C23FE122C23FF93
:102FC4009002E2021E6E790AA2D5205014305209F2
:102FD400B910020404B9080104A2D5205302500117
:102FE40004204F68924FB516005034C0E07F203063
:102FF40050197F30A24F72537252500F123023C2B5
:103004004FC253C252C2557F30800F305203E9C0C1
:10301400E0122C66305203D0E0F9D0E0B516CC3083
:1030240052177F30B9100C122C667F583051077F2D
:10303400788003B90803122C66304F057F2D022CCB
:10304400667F202055F87F2B2053F322924F80CFA8
:103054007F00B40700500B24E2F582E43402F583C8
:10306400E0FF22286E756C6C2900D24E122C23309E
:103074004EF8C24E781630D50108F6022CD22D50E7
:10308400434958122C232403B405004001E4903032
:103094008293122C57743A122C57D250751604028C
:0230A4002EA854
:101DE700E9D2E7C933E833F892D5EDD2E7CD33EC42
:071DF70033FC5002B2D522BB
:101DFE00EC30E7100FBF000C0EBE00080DBD000446
:101E0E000BEB6014A2D5EB13FCED92E7FD2274FFF1
:101E1E00FCFDFEFF22E480F8A2D574FF13FC7D804A
:031E2E00E480EF5E
:101E3100F920E73624F950037907E4F42402FBE59D
:101E410082158270021583DBF6E024FB501BE960EA
:101E510014E4F0E582158270021583E004F0B40AFF
:0D1E610008E4F0D9EE7401F00A22C2D52287
:101E6E00ED33EC3392D5FA602AB4FF33EDC2E77B43
:101E7E00FF60067A1E7993E4227A1E799C20D5049F
:101E8E007A1E7997224E614E002B494E46002D49FF
:101E9E004E4600E47A08F0A3DAFC7B00740722C0F9
:101EAE0083C082ECC0E0EDC0E0EEC0E0EFC0E0EA3F
:101EBE0075F010A4CAABF075F04DA42BFBE435F011
:101ECE00FCEA2410FAEB34C5FBEC34D9FCEDC2E786
:101EDE00FF75F056A4F42411C5F0F434C58FF0A4A8
:101EEE002AE5F03BE43CF020E714122149D0E0FF54
:101EFE00D0E0FED0E0FDD0E0FC12207C8014F40493
:101F0E00122149D0E0FFD0E0FED0E0FDD0E0FC127F
:101F1E001F73D082D083E0FAEDD2E7CD33EC3324B9
:101F2E0082FBE4C3CF33CFCE33CECD33CD33DBF311
:101F3E007B0775F00A846004F0A31B0AE5F0F0A39A
:101F4E008FF0740AA4FFACF08EF0740AA42CFEACD1
:101F5E00F050010C8DF0740AA42CFDE435F0F0A3C2
:051F6E00DBDE74072218
:101F7300EC4D6011E8497017ED33EC3304600DE468
:101F8300FCFFFEFD22E933E8330470F8021E1C1245
:101F93001DE758046009E4CC248150062850090247
:101FA3001E26284003021E23C0E0EB4A7044B9807A
:101FB30006D0E0FB021E12EF4E701CBD8008EBFF43
:101FC300EAFEE9FD80EBE98DF0A4FEE5F002205C7A
:101FD300E9CDF9EAFEEBFFEF89F0A4FCE5F0CE8949
:101FE300F0A42EFFE435F0CD89F0A42DFEE435F006
:101FF3008067EF4E7005BD80D780C3EF8BF0A4AC34
:10200300F0EE8BF0A42CFCE435F0F8EF8AF0A42C6E
:10201300E5F038FCE433CB8DF0A42CFCE5F03BF881
:10202300EE8AF0A42CFCE5F038F8E433CF89F0A471
:102033002CFCE5F038CF3400CE89F0A42FFFE5F077
:102043003EFEE433C98DF0A42EFEE5F039CD8AF0CF
:10205300A42FFFE5F03EFEE43DFD33D0E0FB500747
:102063000BBB000F021E26EC2CFCEF33FFEE33FEFE
:06207300ED33FD021DFE2D
:10207900021E26EC5D046005E859047003021E1C6B
:10208900121DE7580460F6EC4860F2EC7004FDFE9E
:10209900FF22C860DB2481C85009C398600250063A
:1020A900021E239850CAF582E9294B4A7005AB8272
:1020B900021E1275F0007C1A7880C3EF9BEE9AED30
:1020C90099400DC3EF9BFFEE9AFEED99FDE842F0B2
:1020D900DC23ACF0D0E0FFD0E0FED0E0FDAB822005
:1020E900E7101BEB60BAEC2CFCEF33FFEE33FEED8F
:1020F90033FD021DFEE803F830E705C0F075F00076
:10210900EF2FFFEE33FEED33FD40B830E7C280AA72
:102119003F8000004120000042C80000447A0000CE
:10212900461C400047C35000497424004B18968050
:102139004CBEBC205A0E1BCA6753C21C749DC5AE47
:10214900FB60065407601C2323122177EB54386087
:1021590009122163122172121F73ECF8EDF9EEFADC
:10216900EFCB22EB12217280F1543803241C902109
:1021790019FE93FC0EEE93FD0EEE930ECE93FF2205
:10218900BB010689828A83E0225002E722BBFE0254
:09219900E32289828A83E4932287
:1021A200BB010CE58229F582E5833AF583E02250F2
:1021B20006E92582F8E622BBFE06E92582F8E2223C
:0D21C200E58229F582E5833AF583E4932256
:1021CF00BB010689828A83F0225002F722BBFE01EF
:0221DF00F322E9
:1021E100EF8DF0A4A8F0CF8CF0A428CE8DF0A42E12
:0221F100FE22CC
:1021F300BC000BBE0029EF8DF084FFADF022E4CCD0
:10220300F875F008EF2FFFEE33FEEC33FCEE9DEC98
:10221300984005FCEE9DFE0FD5F0E9E4CEFD22EDDE
:10222300F8F5F0EE8420D21CFEADF075F008EF2F28
:10223300FFED33FD4007985006D5F0F222C398FD19
:052243000FD5F0EA22B6
:10224800C5F0F8A3E028F0C5F0F8E5821582700221
:062258001583E038F022BE
:0D225E00EF2BFFEE3AFEED39FDEC38FC22CF
:0E226B00C3EF9BFFEE9AFEED99FDEC98FC226E
:10227900E88FF0A4CC8BF0A42CFCE98EF0A42CFC04
:102289008AF0EDA42CFCEA8EF0A4CDA8F08BF0A482
:102299002DCC3825F0FDE98FF0A42CCD35F0FCEBE1
:1022A9008EF0A4FEA9F0EB8FF0A4CFC5F02ECD39A6
:0F22B900FEE43CFCEAA42DCE35F0FDE43CFC2213
:1022C80075F008758200EF2FFFEE33FECD33CDCCCD
:1022D80033CCC58233C5829BED9AEC99E582984050
:1022E8000CF582EE9BFEED9AFDEC99FC0FD5F0D62D
:1022F800E4CEFBE4CDFAE4CCF9A88222B800C1B957
:102308000059BA002DEC8BF084CFCECDFCE5F0CB94
:10231800F97818EF2FFFEE33FEED33FDEC33FCEBCD
:1023280033FB10D703994004EB99FB0FD8E5E4F988
:10233800FA227818EF2FFFEE33FEED33FDEC33FC75
:10234800C933C910D7059BE99A4007EC9BFCE99A69
:10235800F90FD8E0E4C9FAE4CCFB2275F010EF2FAE
:10236800FFEE33FEED33FDCC33CCC833C810D707AE
:102378009BEC9AE899400AED9BFDEC9AFCE899F8E9
:0E2388000FD5F0DAE4CDFBE4CCFAE4C8F9227C
:10738000C2D5E830E70FB2D5E4C39BFBE49AFAE438
:1073900099F9E498F8EC30E717B2D51273B61223D6
:1073A00004E4C39BFBE49AFAE499F9E498F88003B7
:1073B00012230430D50DE4C39FFFE49EFEE49DFD3F
:0473C000E49CFC222B
:0D239600EF4BFFEE4AFEED49FDEC48FC2246
:0E23A300C3E49FFFE49EFEE49DFDE49CFC224B
:1023B100EB9FF5F0EA9E42F0E99D42F0EC6480C8A3
:0623C10064809845F02243
:1023C700EB9FF5F0EA9E42F0E99D42F0E89C45F06C
:0123D70022E3
:1023D800E8600FECC313FCED13FDEE13FEEF13FFE3
:0323E800D8F12207
:1023EB00E86010ECA2E713FCED13FDEE13FEEF1308
:0423FB00FFD8F022F5
:1023FF00E8600FEFC333FFEE33FEED33FDEC33FC3C
:03240F00D8F122DF
:0C241200E6FC08E6FD08E6FE08E6FF22F6
:0C241E00E0FCA3E0FDA3E0FEA3E0FF2231
:0D242A00E6FB08E6F908E6FA08E6CBF82222
:0C243700E0F8A3E0F9A3E0FAA3E0FB2228
:102443007401FF3395E0FEFDFCA3A3A3E02FFFF08F
:10245300E582158270021583E03EFEF0E582158267
:1024630070021583E03DFDF0E5821582700215834D
:05247300E03CFCF0223A
:0C247800ECF608EDF608EEF608EFF62290
:0C248400ECF0A3EDF0A3EEF0A3EFF022CB
:10249000D083D082E493F608740193F60874029313
:0924A000F608740393F67404734A
:1024A900A8828583F0D083D0821224C01224C0125E
:1024B90024C01224C0E473E493A3C583C5F0C58383
:1024C900C8C582C8F0A3C583C5F0C583C8C582C87D
:0124D90022E0
:0C24DA00A42582F582E5F03583F583220D
:1024E600F8E0FBA3A3E0F925F0F0E582158270027F
:0724F6001583E0FA38F02223
:0924FD00EBF0A3EAF0A3E9F022E0
:10250600D083D082F8E4937012740193700DA3A364
:1025160093F8740193F5828883E473740293686078
:06252600EFA3A3A380DF78
:10252C00EC8EF0A4CCC5F0CCCDF8EFA4CEC5F02D3C
:10253C00FDE43CFCE8A42EC8C5F03DFDE43CFCEFFA
:0D254C00A4FFE5F028FEE43DFDE43CFC2288
:00000001FF
